:1089FA00414952434F5445430056322E342D3033A9
:108A0A0021454E47004241545400424144004032FD
:108A1A0044400040334440004F4646214E455740AB
:108A2A004D454E55000A16000180000300007E00E5
:108A3A0000FE00001E0000360003E60001C400002C
:108A4A0000000FFFE05345415243484053415453FD
:108A5A000043414C40414C544920202300562141B7
:108A6A002152494F2020004241524F4752202000B4
:108A7A00524F555445532020004E454152535420DD
:108A8A0020005741595054532020004D2141215272
:108A9A00214B2320200045584954213F0020202003
:108AAA002141564721202020204453540021455873
:108ABA0049540153454C40524F555445015345546E
:108ACA002048454947485401464C49474854532091
:108ADA006869015741595054532020686901524F1F
:108AEA005554455320206869014149525350414326
:108AFA004568690153455454494E475368690053C0
:108B0A00455420484549474854004241524F40483D
:108B1A004549474854004750532048454947485417
:108B2A00004C4F47424F4F4B20454D505459003E41
:108B3A002145584954002145584954015245504C41
:108B4A0041590153454E440144454C455445002181
:108B5A004558495401544E432031232035374B019F
:108B6A00544E4320312320392E36010150574340B9
:108B7A003130234035374B01505743403130234081
:108B8A0031394B01014D5850403130234035374B74
:108B9A00014D58502034232035374B014D58502071
:108BAA0031232035374B014D585040313023403165
:108BBA00394B014D58502034232031394B014D583F
:108BCA00502031232031394B002145584954014E58
:108BDA00455720205741595054014544495420577C
:108BEA00415950540144454C202057415950540191
:108BFA0001434F4D3A015245434549564520575086
:108C0A000153454E442020202057500153454E44DD
:108C1A0040414C4C4057500101444953542057504D
:108C2A002D57500144454C40414C4C402057500070
:108C3A004252472021444953540053544F5245004D
:108C4A0050524553454E5440504F532E00555044B0
:108C5A004154494E472E2E004044454C4554454404
:108C6A0000574952450049524441004C4953540067
:108C7A0053454E4400205452414E534D49542045C9
:108C8A0052524F52200021455849540153454C45F0
:108C9A004354405255014E4557202020202052501F
:108CAA000145444954202020205255015245564539
:108CBA005253452052550144454C20202020205231
:108CCA00500144454C202020202052550101434F99
:108CDA004D3A01524543454956452052550153459F
:108CEA004E442020202052550053454C21524F55C6
:108CFA005445004E4045405700204E455740504F7E
:108D0A005340210021405245564552534540005296
:108D1A004556525300214044454C40575054530045
:108D2A00214044454C20525445004E4F5420454D55
:108D3A005054592000214053454E44405254450056
:108D4A002145584954014C4F41444043545201561D
:108D5A00494557404354520144454C40414C4C21EB
:0D8D6A0043545201434F4D3A0152454356C8
:108D7700404354520153454E442020435452005619
:108D8700494557204354520020204D4F5645002057
:108D9700204D4F564520544F005343414C4520200A
:108DA700582F5920204558495400205343414C45DA
:108DB7000044495354204B4D0044495354204E4DD1
:108DC70000214558495401564152494F20202068F7
:108DD700690158432D534554202068690147454E82
:108DE7004552414C20686901010154455354464C92
:108DF7004947485401534552564943434F44450157
:108E070042415349432D53455401454153592D532D
:108E170045540021455849540153494E4B212D01D2
:108E270053494E4B404D4F440153494E4B40494ED9
:108E370056015445432020204030304025015641FB
:108E470052205443402020402301564F4C554D4556
:108E570001564152494F204E554C4C004E4F54211C
:108E670050524553454E5400564152494F204E5596
:108E77004C4C004B454550405155494554403130C5
:108E8700404D494E004245464F5245204E554C4CA9
:108E9700494E47002145584954014D4150215452EC
:108EA70041434B014155544F43454E5401545241A0
:108EB700434B2D5550014156472F444953540147C1
:108EC7004C444550415448014C402F4044202020F9
:108ED700202E01535441525401535443594C0153CA
:108EE7005443594C010143594C52002145584954A8
:108EF7000101554E495401434C49434B40302C40E6
:108F0700202301434F4E5452415354014E4D454186
:108F1700213138330040574159504F494E5420456D
:108F270058495354534000574159504F494E5400E4
:108F37002020455849542020210052454345495691
:108F470045004652454540004C4F4144494E472E47
:108F57000053455256494345005341543A004F4642
:108F67004620202020202020200047505320455213
:108F7700524F520053544F52494E472E2E00524FD4
:108F8700555445004E454152455354004C4953549E
:108F9700200045544500414C54403000454D505445
:108FA7005920525445200020544F4F404D554348B7
:108FB7002000214053454C404C4953540020534511
:108FC7004C40575054402100214052454345495693
:108FD7004540002020404F204B40202021004F4B90
:108FE7000020204641494C202021004641494C00A1
:108FF7002045584954004544495400594045405379
:10900700004544495420204E4557202053544F5281
:1090170045005843542D464C494748542000555362
:10902700454400454E54455220004D4D2E4D4D4D63
:1090370020004D4D2753532E5300574753213834A3
:10904700002040554054404D402000554054404D6D
:109057000020555443200053574953534744004178
:109067004C5400535549405800415647003530305D
:10907700003136343000205D203130404B632F7093
:10908700005D2020203140632F2300205D20203504
:10909700404B5453005D203230304046504D005411
:1090A700494D454F555440004C4F43414C00406398
:1090B70040204B63004654204B6300406340204EE2
:1090C7004D004654204E4D004D2F53003230305E38
:1090D700003530305E003122003222003322003565
:0D90E7002200382200464C3700464C31363E
:1090F40000464C333300464C3635004631303000A0
:10910400463136300046323630005E252640534F15
:1091140047005E25264054415300414C54005641BB
:109124005200225E2F24004B545300532F4E002232
:1091340024004B5400225E004E4D00302C3500318B
:109144002C3000322C3000302C3600312C320032DE
:109154002C3500332C3800372C3500403135004095
:109164003330004036300020545241434B214F4E9F
:1091740020200020545241434B214F464620003CBE
:109184002D204C495354202D3E202045584954004D
:1091940053454C004E455854005441534B00464CE3
:1091A4002D4441544500545000544F4600535441FB
:1091B4000046494E004C414E00534554204F46460C
:1091C4005345540049534120484549474854004DAC
:1091D40041524B0020545241434B2D555021200005
:1091E400204E4F5254482D5550212000406A40498A
:1091F4004E20004067404F55540053544152540090
:0992040054502000404F46460082
:1043820075A7049005C2E0F51CE0F51DE0F51EE0FE
:10439200F51FE0F56DE0F56EE0F56FE0F554124FB4
:1043A2003F12497F2275C70375C6E475B901E5BCA2
:1043B200B48143124F3F1259718E628F637568F94F
:1043C200756900124455203C2D203B2B12458A1260
:1043D200455E856D1C856E1D856F1E85541F1244BA
:1043E200C1203C12203243201D2312458A12497FEC
:1043F200E532242850DC221244C1203CF9203DF64B
:10440200203205201DBD80EF301DB880EA12458A9A
:1044120012497F856D1C856E1D856F1E85541F1286
:10442200457412497F203DCE80991247AD201D0D63
:104432007553107400124710203DBB8086E553541B
:104442000FC553C4540F2035051246258003124769
:1044520010808BC23CD23B124511FD124511FC1259
:104462004511C39573F565EC9574F564ED9575602A
:104472000504600A800EE56424E050118006E564BC
:10448200242040091245111245110245111245110D
:10449200FD124511FC124511C39576F567EC95772F
:1044A200F566ED9578600904600122E566F4800204
:1044B200E5668562F0A474E025F04002C23B22C2A8
:0C44C2003C124511A2E7923DA2E6921DBB
:1044CE00A2E592324026A2E492E592E692E7FC1231
:1044DE0045112565F565EC3564F564124511FC1240
:1044EE0045112567F567EC3566F56622A2E492352F
:1044FE00540F79C6F712451109F7301D05124511F3
:10450E00F55322E5697023E56860302402402C24BF
:10451E00FE75F004A485F0C7F5C675B901E5BCB407
:10452E00811985BD68756902801E5403701005C619
:10453E0075B901E5BC056953690F22D23C2214708E
:10454E0004E5BD80F0147004E5BE80E9E5BF80E5AA
:10455E0075A7009006F6E56DF0A3E56EF0A3E56F86
:10456E00F0A3E554F02275A7009006F6E0F56DA3D2
:10457E00E0F56EA3E0F56FA3E0F55422E564B2E733
:10458E00F56D85656EAB67E566FC30E707C3E49BAA
:10459E00FBE49CFCAA62A96312568BE56630E70722
:1045AE00C3E49DFDE49EFEEEB2E7F56F8D542275D9
:1045BE00380C124816124861D553012275380C1268
:1045CE0047E7124857D55301227538001247FF129C
:0F45DE004826D55301227538001247E7124826A8
:1045ED00D5530122753803124816124892D553013E
:1045FD00227538031247E7124888D55301227538C2
:10460D000F1247FF1248B7D553012275380F1247C5
:10461D00E71248B7D553262290462A2373809180FE
:10462D007780688059804A803B802C801D800E8069
:10463D00DA80CB80BC80AD809E808F8080753815F0
:10464D001248161248D9D55301227538151247E76D
:10465D001248CED55301227538091247FF12489FD3
:10466D00D55301227538091247E712489FD55301DA
:10467D0022753806124816124849D553012275384D
:10468D00061247E712483ED55301227538121247DC
:10469D00FF12486FD55301227538121247E71248A1
:1046AD006FD55301220245BD7538151248161248B3
:1046BD00D9D553012275380F1247E71248B7D55394
:1046CD00012275380F1247FF1248B7D553012275D5
:1046DD0038031247E7124888D55301227538031263
:1046ED004816124892D55301227538001247E71229
:1046FD004826D55301227538001247FF124826D59A
:10470D005326229047152373809E80A980B480BFC5
:10471D0080CA80D580E08010801B80268031803C4F
:10472D0080478052805D806875380C1247E71248CB
:10473D0057D553012275380C124816124861D553BE
:0E474D0001227538121247E712486FD553014A
:10475B00227538121247FF12486FD5530122753854
:10476B00061247E712483ED5530122753806124808
:10477B0016124849D55301227538091247E71248DA
:10478B009FD55301227538091247FF12489FD55305
:10479B0001227538151247E71248CED55301220274
:1047AB0046B578C686040886037AED12564978CA50
:1047BB00A60408A60378C686040886037A621256F6
:1047CB004978CCA60408A60378C686040886037A23
:1047DB00B512564978C8A60408A60322751A6A753D
:1047EB001B0A78CA8618088619124A2878CC8606BE
:1047FB000886072278C88618088619E4F51AF51B6F
:10480B00124A2878C886060886072278C6861808B2
:10481B008619751A00751B01024A28E51D2519F525
:10482B001DE51C3518F51CC3E51F9FF51FE51E9EE6
:10483B00F51E22C3E51F9FF51FE51E9EF51EC3E562
:10484B001D9519F51DE51C9518F51C22E51D2FF579
:10485B001DE51C3EF51CC3E51F9519F51FE51E95BF
:10486B0018F51E22C3E51D9FF51DE51C9EF51CC307
:08487B00E51F9519F51FE51E6C
:104883009518F51E22E51F2FF51FE51E3EF51EE5C3
:104893001D2519F51DE51C3518F51C22C3E51D95CD
:1048A30019F51DE51C9518F51CE51F2FF51FE51ED1
:1048B3003EF51E22E51D2FF51DE51C3EF51CE51FEB
:1048C3002519F51FE51E3518F51E22C3E51D9FF5B5
:1048D3001DE51C9EF51CE51F2519F51FE51E351862
:1048E300F51E22E51A7009E51B70058C068D07225B
:1048F300ED851BF0A4A2F792D5ED851AF0A4AEF0D6
:10490300FFEC851BF0A4A2D53FEE35F0FF92D5EC6A
:10491300851AF0A42FFFE435F030D50104FE22E41C
:10492300F51AF51BEF4E7003051B22EF6519700690
:10493300EE65187001227808C3EF33FFEE33FEEF04
:104943009519F5F0EE95184003FEAFF0E51A33F52F
:104953001AD8E5F4F51A751BFF7805C3EF33FFEE9C
:1049630033FEEF9519F5F0EE95184003FEAFF0E531
:024973001B33F4
:10497500F51BD8E5F4C403F51B22E51D9511E51CCF
:104985009510500BE56E9511E56D9510500122E5DA
:104995001F9511E51E9510500BE5549511E56F9582
:1049A50010500122E51D9513E51C9512400BE56E8F
:1049B5009513E56D9512400122E51F9513E51E95AA
:1049C50012400BE5549513E56F9512400122752CA5
:1049D50000C3E51F9554FFE51E956FFE92605007D5
:1049E500C3E49FFFE49EFEC3E56E951DF519E56DD5
:1049F500951CF5189261500BC3E49519F519E495CA
:104A050018F518C3E5199FE5189E9262500AE51836
:104A1500CEF518E519CFF519124922E52C75F003E5
:104A2500A4F538E538904A2E73024A46024A5A02DE
:104A35004A68024A80024A93024AA6024AB4024AD6
:104A4500CC851C16851D17C3E4951FF515E4951E29
:104A5500F514024ADF851C16851D17851E14851F52
:104A6500158077C3E4951DF517E4951CF516C3E489
:104A7500951FF515E4951EF514805FC3E4951DF5A6
:064A850017E4951CF51674
:104A8B00851E14851F15804CC3E4951FF517E495FF
:104A9B001EF516851C14851D158039851E16851F60
:104AAB0017851C14851D15802BC3E4951FF517E482
:104ABB00951EF516C3E4951DF515E4951CF51480AC
:104ACB0013851E16851F17C3E4951DF515E4951C5C
:104ADB00F5148000C3E5179513E516951210D70151
:104AEB0022E5159513E514951210D70122E519F956
:104AFB002517FFE518F83516FED3EF9511EE951037
:104B0B00500122E5119517FDE5109516FC402A4D35
:104B1B0060271248E6E5152FF515E5143EF514E56B
:104B2B00159513E514951210D70122E5199DF9E59A
:104B3B00189CF8851016851117E51729FFE516380F
:104B4B00FEE5139FE5129E500BC3E5139517F9E590
:104B5B00129516F8E51A700AE51B7006AA00AB0150
:104B6B008013E9851AF0A4E5F0FBE8851AF0A42B75
:104B7B00FBE435F0FAE5152BFBE5143AFAE5119B4E
:064B8B00E5109A10D701AD
:104B910022EB9515FDEA9514FCC3E5159511E51475
:104BA100951010D717E5139BE5129A5036E513952A
:104BB10015FFE5129514FE124E5C8027EB9511FF4F
:104BC100EA9510FEAA00C001124E5CD003E5172B36
:104BD100FBE5163AFAEB99F517EA98F516851115E2
:104BE100851014C2D5E5466002D2D5AA56E98AF0ED
:104BF100A4ABF0E88AF0A42B30D50475F00384F857
:104C0100700122E5172513FDE5163512FCED8AF03A
:104C1100A4ABF0EC8AF0A42B30D50475F00384FE2C
:104C2100E5152513FDE5143512FCED8AF0A4ABF072
:104C3100EC8AF0A42B30D50475F00384F9E53890A3
:104C41004C4473024C5C024C68024C71024C7A0277
:104C51004C80024C8C024C93024C98C3743E9EFFD4
:104C6100C3743E99FE8032C3743E9EFFAE0180291B
:104C7100AF06C3743E99FE8020AF06AE01801AC311
:0C4C8100743E9EFEC3743E99FF800EC37B
:104C8D00743E99FF8007C3743E9EFEAF0108EF246A
:104C9D0037FFE51B7007E51A700CE8800EA2E7E5FB
:104CAD001A50030460F488F0A4E5F0600104F923C0
:104CBD00FA98FBC3E998C333F9904CCCE5387302ED
:104CCD004CE4024D11024D46024D73024DA0024DB2
:104CDD00CD024DFA024E2705A7800BEB30E7032AD4
:104CED008002291E1FFBEEC45403F583EE5408C445
:104CFD002FF582EE5407243883F5F0E045F0F0D817
:104D0D00DA05A72205A7800BEB30E7032A800229DD
:104D1D000E1FFBEEC45403F583EE5408C42FF58229
:104D2D00EE5407240B83F5F0E045F0F0D8DA05A733
:104D3D0022804020100804020105A7800BEB30E70C
:104D4D00032A8002291E0FFBEEC45403F583EE5493
:104D5D0008C42FF582EE540724EC83F5F0E045F0FE
:104D6D00F0D8DA05A72205A7800BEB30E7032A80E0
:044D7D0002290E0FEA
:104D8100FBEEC45403F583EE5408C42FF582EE54B0
:104D91000724BF83F5F0E045F0F0D8DA05A7220536
:104DA100A7800BEB30E7032A8002291F1EFBEEC40C
:104DB1005403F583EE5408C42FF582EE5407249270
:104DC10083F5F0E045F0F0D8DA05A72205A7800BBE
:104DD100EB30E7032A8002291F0EFBEEC45403F5D2
:104DE10083EE5408C42FF582EE5407246583F5F051
:104DF100E045F0F0D8DA05A72205A7800BEB30E7F4
:104E0100032A8002290F1EFBEEC45403F583EE54DE
:104E110008C42FF582EE5407243883F5F0E045F0FD
:104E2100F0D8DA05A72205A7800BEB30E7032A802B
:104E310002290F0EFBEEC45403F583EE5408C42F70
:104E4100F582EE5407240B83F5F0E045F0F0D8DA53
:104E510005A7228040201008040201EC701FED20FC
:084E6100E740D2E023CF23CF8C
:104E690030E7F980357B08801A7B1080167B20801B
:104E7900127B40800E20E4ED20E3EE20E2EF20E1FA
:104E8900F07B80EE8BF0A4CF8BF0A4E5F02FFFEC44
:104E99008BF0A4CD8BF0A4E5F02D2499838FF0A499
:104EA90033E5F033FBE98BF0A4E5F0C88BF0A428D7
:104EB900F9E435F0F822FFFEFCFAF8F6F4F2F0EF27
:104EC900EDEBEAE8E6E5E3E1E0DEDDDBDAD9D7D6CA
:104ED900D4D3D2D0CFCECCCBCAC9C7C6C5C4C3C11F
:104EE900C0BFBEBDBCBBBAB9B8B7B6B5B4B3B2B131
:104EF900B0AFAEADACABAAA9A8A8A7A6A5A4A3A319
:104F0900A2A1A09F9F9E9D9C9C9B9A9999989797D7
:104F1900969594949392929190908F8F8E8D8D8C7B
:104F29008C8B8A8A89898887878686858584848304
:104F390083828281818075A700904F65E546FA24B6
:104F4900FA50027A05EA2323F978107F0493F608C8
:104F590009E9DFF9904F7DEA93F556227FC2803E39
:104F69007F4680BA7E8C81747D1882E87A3085D03C
:104F790074608BA0808040201008124F890251DD97
:104F8900D215D234D274D273C219C23A1259718E5F
:104F990047757D00754605755202127ED6120203C9
:104FA900E53524E25003127ED6E55275F016A4F5D4
:104FB900701251937551151250577F237E09908DA8
:104FC9008F1265E212C5AF10000810010D10021210
:104FD90080E212510675330180DA12514B753301A3
:104FE90080D27551001250577E00908DA01266151F
:104FF9007F237E05908D961265E21250AF12C5AFE0
:10500900E55210000F10010510029280D5045403D7
:10501900F55280CE1250577F237E0B908DB11265C9
:0F502900E2E54660071460041412348112C5AF2B
:10503800E54610000810010B10021180D860D61543
:105048004680D2B4050280CD054680C9024FA675B8
:10505800320012C7657F017E11908D861266157F1A
:105068002F7E0090BECB12BCB37E3C90BECB12BC50
:10507800B3E55112BE6A75170812C1AD1234B17585
:10508800710012C103741BFFF5177E0F908DB830A5
:105098005D03908DC0126615127F19125F011238D8
:1050A800C41243A70212F4E552601414601E14607F
:1050B800297F647E2D791C1250F91E1FD9F9227F91
:1050C8006A7E1F79281250F91FD9FA227F487E2D4F
:1050D800791C1250F90F1ED9F9227F567E33792890
:1050E8001F12C6AA0F0F12C6AA1F12C6AA1ED9F0EF
:1050F800221E12C6AA0E0E12C6AA1E02C6AAE55281
:10510800605514606814606D800075709E1251803F
:105118008003757000E5732540F573E43574F57404
:10512800E43575F5752275701612511D800375707A
:105138002DE5762542F576E5773541F577E435783E
:10514800F57822E55260CB1460DC1460E1800075CC
:105158007044125139800375705AE5739540F573A0
:0C516800E5749400F574E5759400F5758D
:10517400227570711251628003757088E5769542CC
:10518400F576E5779541F577E5789400F57822E5AD
:10519400469051A993F540FEAD47E4FFFC12571E1B
:1051A4008E418F4222020C183060C07F37120705EF
:1051B40012130A12C5AF12548BEB7005908B328018
:1051C4000B12526A908FDA5003908FE87F367E0478
:1051D4001265E212C5AF12C67AE4F535F5207537CB
:1051E40009908D4A1212069051EF7302027B02530A
:1051F400B7024F830254BC02520402521D0251AF43
:105204007F25120C1C80D27F2D7E04908FAE1265F8
:10521400E212C5AF12C67A80C07F2E1207051213A0
:105224000A12C5AF12546F123A46D2AC1000AA301B
:105234006DFA12531A203BCF40ED7568F9751600CC
:1052440012536A40FB1255297F2E7E35E51612BB98
:10525400F112C5AF051612668878C6B6F7E2125485
:10526400D87F2D02545E7C03123A4612C345744122
:1052740012C378745312C313EB12C33412669A50D8
:1052840003DCE5227515F975160010000EE51560AE
:10529400251252BC40051252E35002D3227F367EBF
:1052A40029E51612BB3A12C5AF7F1412C691051632
:1052B400E51664F870D4C322126C1375B901E5BC09
:1052C400B4811AE5BDF51570037516F778C6A616F0
:0952D400126D5C126D54126D5450
:1052DD00C3026D54D3227F0375F019D5E0FDD5F0CF
:1052ED00FA123A4612C345744112C378744212C37E
:1052FD00137E0F78C6E60812C313DEF912C33712F8
:10530D00669A400122DF012275F00080CEC23B1269
:10531D003A46D2AC12C4B9C5F0603EC5F0B440F403
:10532D0012C4BEB4400312C4BEB4412DF53812C42C
:10533D00BEB4532512C4BEFA12C4BEE538701A129B
:10534D00C4BEB40D1412C4BEB40A0EC3E5169A4001
:10535D000302667FC2ACD23B22C2ACD3221266DD01
:10536D00123A46D2AC1000F112C4B9C5F060EAC5CC
:10537D00F0B440F112C4BEB4400312C4BEB441D95E
:10538D00F53812C4BEB442D17E1078C612C4BEF632
:10539D0008DEF9E53870C212C4BEB40DBC12C4BE2D
:1053AD00B40AB6C2ACC3220251DD7F0A1207051240
:1053BD00130A12C5AF12546F123A98D2AC1000E70F
:1053CD0012C4BEB440F5F53812C4BEB46EED12C4AD
:1053DD00BEE538600A123A98744F12C31F80DC7F05
:1053ED000A7E35E51612BBF112C5AF12C373E51671
:1053FD0012C31F12C3297568F9751600123A98D297
:10540D00AC10005B12C4BEB440F7F53812C4BEB484
:10541D004EB97E1078C612C4BEF608DEF9123A985F
:10542D00E5386007744F12C31F80D1125529051638
:05543D00745112C31FB1
:1054420078C6B6F7C21254D812C6817F0A7E35E5F5
:105452001612BBF112C5AF12C6817F097E35908F3D
:10546200E51265E212C5AF12C67D0251DD75150067
:10547200751605126C0A75B901E5BC30E70205160E
:105482000515E515242050EB227B007515F9126CE9
:105492001375B901E5BCB481010B0515E5152402AC
:1054A20050EC751501126C0A75B901E5BCB48101A5
:1054B2000B0515E515242050EC227F1C120705125E
:1054C200134D12C5AF10000B10010280F87515F9CB
:1054D2001254D80251DDE51560372402401A241E09
:1054E2005019E515240740028027126C1312551437
:1054F2000515E515240250F2751501126C0A75B9ED
:1055020001E5BC30E7031255140515E515242050BA
:10551200EA2212A65512408905C612408905C61212
:10552200408905C6024089E568606AF5150515E5FA
:10553200152402501D751501126C0A75B901E5BCDE
:1055420030E70280190515E515242050EB7515008A
:10555200800C241E60F750E0E51524065037E568FC
:1055620075F004A485F0C7F5C675BC81E515F5BDD7
:10557200F56878C6B6F70375BD000812558C12554A
:105582008612558686BC0886BD0886BE0886BF0878
:0655920012408905C6224B
:10AB00001299DF12ABFF12712612AB8412712E1252
:10AB1000AB910299E31299DF12ABFF1271267F5AB3
:10AB2000C23C127008127204783F79437F607EEA5B
:10AB300012ABF312712E7F65127008127204783D09
:10AB400079417F207E4E12ABF3303C2012ADB5121E
:10AB5000AC10783F794312AB6F783D794112AB6FFF
:10AB600012ADB578D7E65480F67537000280EBC396
:10AB7000E796FF1819E796FE0809C3E69FF718192C
:10AB8000E69EF7227F5B7E0690906A1266151F8014
:10AB90000A7F667E14745912BC531F126E917E395F
:10ABA000E402BC727866E620E73418C3E6947208C3
:10ABB000E694045029C318E6941F08E69404401E46
:10ABC0007869E620E71818C3E6940E08E694015069
:10ABD0000DC318E6947508E694004002D322C32200
:10ABE000E67D0030E7011D08E62BFB18E63CFCE49F
:0EABF0003DFD22C3EB9FF6F71819EC9EF6F719
:10ABFE002212ABA4400CE47842F608F67840F60830
:10AC0E00F6227864C3E6946AF55708E6944CF55636
:10AC1E000808C3E69458F55B08E694AEF55A753904
:10AC2E0000AC56AD57EC129D8C784C129E1AAC5A55
:10AC3E00AD5BEC129D8C7850129E1A7F2B7E867D1A
:10AC4E00777C18129D517850129E0E129C5D129DAB
:10AC5E00517850129E0E129C5D129D517850129E8C
:10AC6E000E129C5D129D517F367E847D257C641272
:10AC7E009D517850129E0E129C5D129D51784C1271
:10AC8E009E0E129C5D129D517F3F7EA27D607C8B3D
:10AC9E00129D517850129E0E129C5D129A4B129A72
:10ACAE004B129E267F3F7E807D057CE60539129CE9
:10ACBE005D7848129E1A7F2C7E937D477C7F129D75
:10ACCE00517850129E0E129C5D129D517850129E1C
:10ACDE000E129C5D129D51784C129E0E129C5D12AE
:10ACEE009D517F357EB47DF87CDF129D51785012D8
:10ACFE009E0E129C5D129D517850129E0E129C5DFE
:10AD0E00129D517F3F7EED7D227CCD129D51784C60
:10AD1E00129E0E129C5D129A4F129A4B7844129EFE
:10AD2E001A7F317E397D9D7CE7129D51784C129EA3
:10AD3E000E129C5D129D51784C129E0E129C5D124D
:04AD4E009D51784457
:10AD5200129E0E129A4F129D517F2C7E377D0C7CD3
:10AD6200A3129D51784C129E0E129C5D129D517839
:10AD72004C129E0E129C5D129D51784C129E0E1228
:10AD82009C5D129A4F129E267F3F7E807D027C9FA1
:10AD92000539129C5D7844129E1A7848129E0E1252
:10ADA2009DC38E428F437844129E0E129DC38E40E5
:10ADB2008F4122753900AC42AD43EC129D8C78482C
:10ADC200129E1AAC40AD41EC129D8C7844129E1A30
:10ADD2007F2B7E537D507C09129D517848129E0E26
:10ADE200129C5D129D517848129E0E129C5D129D1E
:10ADF200517844129E0E129C5D129D517F347EF258
:10AE02007DCD7CA3129D517848129E0E129C5D123C
:10AE12009D517848129E0E129C5D129D517F3F7E7D
:10AE22000A7D2E7CAE129D517844129E0E129C5DBC
:10AE3200129A4B129A4B784C129E1A7F2B7E4F7DA0
:10AE4200AF7CB2129D517848129E0E129C5D129DEB
:10AE5200517848129E0E129C5D129D517848129EA6
:10AE62000E129C5D129D517F357EB17D4B7C9512F9
:10AE72009D517848129E0E129C5D129D517844128B
:10AE82009E0E129C5D129D517F3F7E497DCD7C4579
:10AE9200129D517848129E0E129C5D129A4F129A80
:10AEA2004B7850129E1A784C129E0E129DC38D55ED
:10AEB2008E568F577850129E0E129DC38D598E5A00
:04AEC2008F5B7864C6
:10AEC600E557246AF608E556344CF608E555340489
:10AED600F608E55B2458F608E55A34AEF608E4357C
:03AEE60059F622F8
:107F39001299DF1285CA1299E37F669090521266F0
:107F490013127FA77F5A78C4127F83127F8B78C65A
:107F5900127F83127F6E7F6578C8127F83127F8BB1
:107F690078CA127F837E2DE51B12BC727E33E51A17
:107F790012BC727E39E51902BC72860408860302B6
:107F890055E87E15E51C12BC727E1BE51B12BC72FE
:107F99007E21E51A12BC727E27E51902BC727F5A4E
:107FA9007E01E53A12BB887E0B9089BEE53B9302C0
:107FB900BC85E6FF08E6FE08E6FD339217E45001AA
:107FC900F4FC129E3775130A75390112A03578D75A
:107FD900E6C2E775F00A84F9303D02A9F0129E372E
:107FE9008913053912A00E30170A053912A0210587
:107FF9003912A021A803029E1A1299DF1285CAC25A
:108009003C7F5A7E031273B5127FA712C5AF1000C9
:108019000810011510022080EFE53A146004153AA2
:108029008003753A3CD23C80DFE53AB43C05753AA9
:108039000180F2053A80EE7E031273B07E0B127353
:10804900B5127FA712C5AF10000810011510022044
:1080590080EFE53BB40205753B158002153BD23C28
:1080690080DFE53BB41505753B0280F2053B80EEE8
:108079007E0B1273B07F5A78C4127F83127F8B12E2
:0780890080F412721478C4A8
:1080900012814C78C6127F83127F6E128126751C66
:1080A0000012721478C612814C7F6578C8127F83E3
:1080B000127F8B1280F412721478C812814C78CA25
:1080C000127F83127F6E128126751C001272147843
:1080D000CA12814C303C14E53B24F4500B78C9E6BD
:1080E0002410F618E63427F61281521299E3126D25
:1080F0009602C5AFC2247E15E51C127305F51CD28D
:10810000247E1BE51B127305F51B1023E77E21E57A
:108110001A127305F51A1023E67E27E51912730566
:10812000F5191023E822C2247E2DE51B127305F5F4
:108130001BD2247E33E51A127305F51A1023E77E4D
:1081400039E519127305F5191023E622ECF608EB50
:10815000F6221289D678C8E6FE0886073395E0FD38
:10816000FC129D517FE87E037D007C0012A0351239
:108170009D5178CAE6FE0886073395E0FDFC12A003
:108180000E129D517F807E697D677CFF12A00EECF0
:10819000129D88129D517F3F7E807D0D7C1D129C1B
:1081A0005D129D517F3D7E407D007C00129D517887
:1081B000BC129E0E129C5D129D517F3E7E807D0002
:1081C0007C00129A4F129D5178BC129E0E129C5D3B
:0981D000129D517F3F7E807D006D
:1081D9007C00129A4B129D5178B4129E0E129C5D2E
:1081E900129CD5783C129E1A7F407E807D007C00CF
:1081F900129D51783C129E0E129C5D129EB4129DE6
:10820900517F3F7EA87D007C00129D5178B8129E57
:108219000E129C5D129C5D129D517F407E007D0077
:108229007C00129D51783C129E0E129C5D129EB4E8
:10823900129D517F3F7EC07D007C00129C5D129A89
:108249004F129D5178B8129E0E129C5D129D517865
:108259003C129E0E129A4F7854129E1A129E9E78C4
:1082690058129E1A129D51129C5D129D5178C0128E
:108279009E0E129C5D7844129E1A7854129E0E121C
:108289009EB4783C129E1A129D51129C5D129D510A
:1082990078BC129E0E129C5D783C129E1A7F3E7E1F
:1082A900C07D007C00129D51783C129E0E129C5D8F
:1082B900129D517F3F7E007D007C00129A4F129DD6
:1082C90051783C129E0E129C5D129D517F3F7E801B
:1082D9007D007C00129A4F129D5178B4129E0E12A5
:1082E9009C5D7870129E1A78C4E6FE08860733955D
:1082F900E0FDFC129D517FE87E037D007C0012A009
:1083090035129D5178C6E6FE0886073395E0FDFCD7
:1083190012A00E129D517FE07E5E7DF87CFF12A0B7
:108329000EEC129D88129D517F3F7E7F7DE57CC9B1
:05833900129D51787057
:10833E00129E0E129C5D129CD57850129E1A7F3F93
:10834E007EF07D007C00129D51783C129E0E129C98
:10835E005D129D517F3F7EC07D007C00129A4F12B0
:10836E009D51783C129E0E129C5D129D517F3F7E58
:10837E00807D007C00129A4F783C129E1A78BC12B7
:10838E009E0E129D517F3F7E807D007C00129A4B87
:10839E00129D51783C129E0E129D5178B4129E0E73
:1083AE00129C5D129C5D7840129E1A7854129E0E9D
:1083BE00129EEC783C129E1A129D51129C5D78749E
:1083CE00129E1A7F417E107D007C00129D5178C056
:1083DE00129E0E129C5D129D517F407E807D007C10
:1083EE0000129D517844129E0E129C5D129D517F7B
:1083FE00417E207D007C00129A4B129D51784412D2
:10840E009E0E129C5D129D517F407E407D007C0031
:10841E00129D517874129E0E129C5D129D517F40DA
:10842E007EA07D007C00129A4F129A4F129A4B1228
:10843E009D517850129E0E129C5D129D51785012D5
:10844E009E0E129C5D129D517F3D7E2A7DAA7CABB5
:10845E00129C5D129D517F3F7E007D007C00129A22
:10846E004B129D51783C129E0E129D517870129EA9
:10847E000E129C5D129D517840129E0E129CD512CA
:10848E009D517850129E0E129C5D129D5178501285
:10849E009E0E129C5D129C5D129D517854129E0E82
:0C84AE00129A4B129D517F4A7E517DD2E4
:1084BA007CCB129C5D129DC378AC129E1A7F407EC3
:1084CA00007D007C00129D517874129E0E129C5DF4
:1084DA00129D517F3F7E807D007C00129A4F129D33
:1084EA00517844129E0E129A4F129D517850129E44
:1084FA000E129C5D129D517850129E0E129C5D12B6
:10850A009D517850129E0E129C5D129D517F3E7EA7
:10851A002A7DAA7CAB129C5D129D517850129E0E48
:10852A00129A4B129D517858129E0E129CD5129D8A
:10853A00517F4A7E517DD27CCB129C5D129DC31223
:10854A009D51AF3AEF3395E0FEFDFC129D517F40FD
:10855A007E7E7D057C0012A035129D517F607E755E
:10856A007D587CFF12A00E12A00E78B0129E1A78C7
:10857A00AC751B641285A18F1C78B0751B671285B8
:10858A00A1E51C75F00AA42FFF249C50027F0078F5
:10859A00D7E654802FF622753900129E0E129D518D
:1085AA007F0A7E007D007C0012A0E1A81BE513F67D
:1085BA0008E512F608E511F6335004EFF404FF2239
:1085CA00C23D78647BAC127FBBD23D78677BB01228
:1085DA007FBB1289D67F007EE47D577C00129D51B5
:1085EA0078AC129E0E12A00E129D517F007E537D12
:0E85FA00077C0012A0E1129D7085133B7F806C
:108608007ECB7DA47C00129D5178B0129E0E12A0E4
:108618000E129D517F407E7E7D057C0012A0E112E6
:108628009D70E513F56F04F53A85126E85116D8519
:10863800106C7F407E7E7D057C00129D51786C1207
:108648009E0E12A035129D517F607E0C7DA27C008B
:10865800129D5178B0129E0E12A00E12A021786CB5
:10866800129E1A78AC129E0EEC129D88129D517FB4
:10867800347E9C7D2B7C5F129C5D7854129E1A126E
:108688009E9E7850129E1A786C129E0EEC129D884F
:10869800129D517F347E9C7D2B7C5F129C5D129DC8
:1086A800517850129E0E129C5D7840129E1A7F409F
:1086B8007E007D007C00129D517854129E0E129C03
:1086C8005D129EB4129D517F3D7EC07D007C0012DC
:1086D8009D5178BC129E0E129C5D129D517F3E7E6C
:1086E800C07D007C00129A4F129D5178BC129E0EDC
:1086F800129C5D129C5D129D517F3D7E407D007CE9
:1087080000129D5178BC129E0E129C5D129D517FE5
:108718003E7E807D007C00129A4F129D5178BC12DB
:108728009E0E129C5D129D517F3F7E807D007C00D5
:10873800129A4B129D517854129E0E129C5D129AF9
:108748004B129D517F407E807D007C00129D5178A8
:1087580054129E0E129C5D129EB4129D517F3D7E56
:10876800707D007C00129D5178BC129E0E129C5D9B
:10877800129D5178BC129E0E129C5D129C5D129A3D
:108788004F129D5178B4129E0E129C5D7858129E1D
:108798001A7854129E0E129EB4783C129E1A78547F
:1087A800129E0E129EEC7854129E1A783C129E0E5F
:1087B800129D51129C5D129D5178BC129E0E129C06
:1087C8005D783C129E1A7F3E7EC07D007C00129D23
:1087D80051783C129E0E129C5D129D517F3F7E0087
:1087E8007D007C00129A4F129D51783C129E0E1209
:1087F8009C5D129D517F3F7E807D007C00129A4FC8
:10880800129D5178B4129E0E129C5D7870129E1AB9
:108818007850129E0E129D51129C5D129D5178C087
:10882800129E0E129C5D7844129E1A7854129E0E67
:10883800129D51129C5D7874129E1A7840129E0EF9
:10884800129D51129C5D783C129E1A7F407E807D5D
:10885800007C00129D517844129E0E129C5D129D60
:10886800517F417E107D007C00129A4F129D5178F5
:1088780044129E0E129C5D129D517874129E0E1227
:108888009D517F407EA07D007C00129A4B129A4F2A
:10889800129D51783C129E0E129C5D129D517F3D97
:1088A8007E2A7DAA7CAB129C5D129D517F3F7E0083
:1088B8007D007C00129A4F129D517854129E0E1220
:1088C8009D517870129E0E129C5D129D51783C123B
:1088D8009E0E129C5D129C5D129D517858129E0E40
:1088E800129A4F129D517F3F7E7F7DE57CC9129C75
:0188F8005D22
:1088F900129D517F4B7E187D967C80129A4F129D56
:10890900C3129D517FE87E037D007C0012A0E11215
:108919009D7078C8A61208A61308A60608A60778A7
:1089290074129E0E129D517F3F7E807D007C001245
:108939009A4B129D517844129E0E129A4F129D51D4
:108949007F3E7E2A7DAA7CAB129C5D129D517840A8
:10895900129E0E129C5D129D51783C129E0E129C25
:108969005D129D517840129E0E129A4F129D517FB1
:108979003F7E7F7DE57CC9129D517870129E0E1253
:108989009C5D129C5D129D517F487EF47D247C0084
:10899900129A4F129DC3129D517FE87E037D007C80
:1089A9000012A0E1129D7078C4A61208A61308A6A9
:1089B9000608A607223F3F4344454647484A4B4CD1
:1089C9004D4E5051525354555657583F3FE4F5397F
:1089D900F5A79089EA791078B4E493F6A308D9F950
:1089E9002232A5C24A4A19DC3A885CDB3BFFD6DC55
:0189F9003B42
:1099DF00D2D58002C2D575A70490040078107F0BF2
:1099EF00129A0B78267F05129A0B783C7F22129AD7
:1099FF000B786A7F0F129A0B75A7002230D506E6F7
:109A0F00F008DFFB22E0F608DFFB22D2D58002C28E
:109A1F00D575A7049006FA78737F06129A0B75A76F
:109A2F000022DA0CD902800BD906303701B350056A
:109A3F00029BBE9237029BAAD9F680F9D2368002DA
:109A4F00C236129BEF303606C86002B237C8923664
:109A5F00DAD0D9E4B8000A129C36A2369237029BAC
:109A6F009360FBB51300400F129C36A23692F7A2FB
:109A7F00379236A2F79237C398F40424E740DF24D5
:109A8F0019AD29AC28AB277A00C394084008CDCC78
:109A9F00CBCAE4CD80F424086010F9C3ED13FDECBC
:109AAF0013FCEB13FBEA13FAD9F1A236303701B3EB
:109ABF0040308A17E5102BF518E5113CF519E51222
:109ACF003DF51A501A13F51AE51913F519E5181380
:109ADF00F518E51713F5170513E5137002051402B2
:039AEF009B49E4AC
:109AF200C39AF517E5109BF518E5119CF519E512C7
:109B02009DF51A500DB237C378177F04E496F60814
:109B1200DFFA7A047019E513C39408F5135002159D
:109B220014E4C517C518C519F51ADAE8029BEA202C
:109B3200E7BAE5137002151415137817C37F04E60C
:109B420033F608DFFA80E8E51A20E7137817C37FB7
:109B520004E633F608DFFAE513700215141513E56F
:109B6200173378187F03E63400F6500E08DFF775D6
:109B72001A800513E51370020514E51420E75470EA
:109B820027E513604E046020851A12851911851885
:109B9200105326F0AC10AD11A237E51313FFE512F6
:109BA20092E7FEA813029D70E4F512F511F510F587
:109BB200147513FF5326F043260580D8E5FFF512EE
:109BC200F511F510751400F513D2375326F043261C
:109BD2000980C15326F0432603E4F512F511F5106E
:109BE200F514F513C23780AC5326F080EC79017A74
:109BF200018512F0E513A2F7339237751400F513BD
:109C02006002D2F785F012A813B8FF0809E512C264
:019C1200E76A
:109C13006001098C278D288EF0A2F7EF3304700AB8
:109C23000AC2F705F00AD5F0011A146002D2F785CB
:109C3300F02922C88813C512C529C512C511C52824
:109C4300C511C510C527C51022DA03B80003029B4E
:109C5300BED9028002D9F7029BAA129BEF303701CB
:109C6300B392377004D9E78005DADEB80003029BAC
:109C7300EAD9E2C3947E500215142513F51350025A
:109C830005147815760008B81BFA78277915E608C5
:109C9300FAE8FC78108AF0E608A427F709E5F0371C
:109CA300F7500989F00907E760FBA9F0B813E61933
:109CB30019ECF8B82AD8029B49029BD5B8FFFA02DF
:109CC3009BBED9FB029BAADAF6B800F0029BEA120C
:109CD3009E26129BEF303701B392377007D9E3B852
:109CE30000E280DBDAE1B8000280E1D9D5C8C3988D
:109CF30050021514247F50020514F513781A7600C8
:109D03007A1A7B80C3E5109527E5119528E512950E
:109D1300294016C3E5109527F510E5119528F5118F
:099D2300E5129529F512E64BF654
:109D2C00DA03029B49EB03FB30E703187600C3E52B
:109D3C001033F510E51133F511E51233F51240CA65
:109D4C0030E7DD80B6E53905396010D0F0D0E0C0E1
:109D5C0010C011C012C013C0E0C0F08F138E128D52
:109D6C00118C1022E539146010D0F0D0E0D013D053
:109D7C0012D011D010C0E0C0F01539227920800C1F
:109D8C007910800479087D007E007F003392D550D5
:109D9C0003129E00EC33400FEF33FFEE33FEED3336
:109DAC00FDEC33FCD9EE22EECCF5F0747E29A2D575
:109DBC0013FF92F7AEF022EF8EF0A2F7D2F73392A8
:109DCC00D5C3947F5006E4FFFEFDFC229420400492
:109DDC0074FF80F304CCFEE4FFFAE5F0CC6012C310
:109DEC00CC13CCCD13CDCE13CECF13CF0450EEDA93
:109DFC00EC30D5D7C3E49FFFE49EFEE49DFDE49CCC
:039E0C00FC22E64F
:109E0F00FC08E6FD08E6FE08E6FF22ECF608EDF694
:109E1F0008EEF608EFF622CFC513CFCEC512CECD82
:109E2F00C511CDCCC510CC22E4F513F512F511F503
:109E3F001022E493FCA3E493FDA3E493FEA3E49325
:109E4F00FFA322C0E0129D51129C5D129E85129EAF
:109E5F0041D0E0C0E0129D51129E7C129C5D129D7C
:109E6F0051129E41129A4FD0E0D5E0E722AC48AD97
:109E7F0049AE4AAF4B228C488D498E4A8F4B227484
:109E8F00FF7809FFFEFDFCE52654F048F526221267
:109E9F009F4504A2E1927F1420E015909FC67404A1
:109EAF00129E528029129F4530E102B27F20E0EBD3
:109EBF008C4C8D4D8E4E8F4F909FDA7404129E52A4
:109ECF00129D51AC4CAD4DAE4EAF4F129C5D307FDD
:109EDF0004EF6480FFEE33EF337001FF22129F45D2
:109EEF00C0E08C4C8D4D8E4E8F4F909FFE740312A1
:109EFF009E52129D51AC4CAD4DAE4EAF4F129C5D6C
:019F0F00EC65
:109F1000C54CFCEDC54DFDEEC54EFEEFC54FFF90A7
:109F20009FEE7403129E52D082129D51AC4CAD4DE7
:109F3000AE4EAF4FE58230E007129CD5B27F809DD8
:109F4000129CD28098EE33EF3324605007D0E0D0DB
:109F5000E0029E8EEFA2E7547F927FFF129D517C1C
:109F6000837DF97E227F3E129C5DEE33EF332481A8
:109F70005010129D51129DC3129D88EFB2E7FF123F
:109F80009A4FEE33EF33602A2403F8C313FFEE92A7
:109F9000E7FEE82481E4501A129D51129DC3EF049C
:109FA000C2E0FCF582129D90EFB2E7FF129A4FE5F6
:109FB0008203FAEE33EF33600B148FF0A2F713FF36
:109FC000EE92E7FEEA2283FA703AE4E9AABCF8E0EE
:109FD000813EE6E99DBF0000803F1A3C2839666952
:109FE00099BBE335A33DE75D25BFDB0FC93FCCDB64
:109FF0008D41EE3649C43F91C9453DF8B0C50000DA
:10A00000803F34F517C373FA2F45DDFD0AC6EF25EF
:10A0100013FFEE3512FEED3511FDEC3510FC029DFF
:10A0200070C3EF9513FFEE9512FEED9511FDEC95C3
:10A0300010FC029D70EFF88513F0A4FFE513C5F046
:0AA04000CEF9A42EFEE435F0CDFAAF
:10A04A0088F0E512A42EFEED35F0FDE433CC85133D
:10A05A00F0A42CFCE5128AF0A42CFCE51189F0A4EA
:10A06A002CFCE51088F0A42CFC89F0E512A42DFD47
:10A07A00EC35F0FCE51188F0A42DFDEC35F0FC8AF6
:10A08A00F0E513A42DFDEC35F0FC029D70E4CCF84C
:10A09A00E4CDF9E4CEFAE4CFFB75F020C3E513333F
:10A0AA00F513E51233F512E51133F511E51033F521
:10A0BA0010EF33FFEE33FEED33FDEC33FCEF9BEE96
:10A0CA009AED99EC98400CFCEF9BFFEE9AFEED9905
:10A0DA00FD0513D5F0C622C2D5EC30E705B2D5127C
:10A0EA009E00E51030E70DB2D512A10412A0971216
:10A0FA009E00800312A09730D515C3E49513F5137B
:10A10A00E49512F512E49511F511E49510F5102273
:10920D00E57124885002D2191259718E47127F19B7
:10921D00125D02305E0F125CA01276A9125BF31282
:10922D00AA5D123539122D6E123A00103626301203
:10923D0019E412934812935D12945F129481305188
:10924D000302950B1297DC205109C251E4F552F53A
:10925D0045F5442274FF1293481259718E1C8F1BD1
:10926D007510DF751100E51164B470061293137556
:10927D0011101292E04028AE1CAF1B1259F720328C
:10928D001EAC03AB027A0C125620ED701275A700BE
:10929D00758304851182ECF00583E510F00511D579
:1092AD0010C412931375C70375C6E075A704900516
:1092BD00007F041292CEDFFB75A700122010025C16
:1092CD00A0E0F5BCE0F5BDE0F5BEE0F5BF124089CC
:1092DD0005C622E51075F004A4F5C685F0C775B96D
:1092ED0001E5BC33401F05C605C675B90185BE64D1
:1092FD0085BF6505C675B90185BC6685BD6785BE2B
:10930D006885BF69C322E51124FE502E75A7007F25
:10931D0010AE111E7583048E82E0FD1582E0CDB571
:10932D0005005012F00582CDF00583E0FD1582E0B9
:10933D00CDF00582CDF0DEDCDFD72275A754900489
:08934D000005A79005007FB4A4
:10935500F0F0DFFC75A7002212A8A9C2517B077A9D
:10936500FFE4FFF5A7900400129443ED244C40352B
:10937500EC603075A7008D8205A7129409758305E9
:109385008D82E02410401CF005A7E02CF050050567
:10939500A7E004F0BA000CBB0009D251EF24DC5061
:1093A500027F23DFC3EA60051293BC8006EB6003EE
:1093B5001293F475A7002230E0047553082230E1BA
:1093C500047553182230E2047553282230E30475DE
:1093D50053382230E4047553482230E50475535858
:1093E5002230E6047553682230E70375537822303E
:1093F500E0047553882230E1047553982230E20366
:109405007553AA22ED54F0C4232390941373530289
:10941500FE225302FD225302FB225302F72253027E
:10942500EF225302DF225302BF2253027F2253034E
:10943500FE225303FD225303FB225303FB2212A7F3
:10944500B212A6B5E4F5F7C2B2C2B2ADF7F5F7C2EE
:10945500B2C2B2ACF7D2B2C2202290050078B4E015
:109465006015FD54F0C4CD7C00540FFE1583E0FF5C
:0594750012571EEFF08C
:10947A0005830582D8E42275830478FF088882E090
:10948A0060FAF5D38812E512244C50012285D3D212
:10949A0088D4881279FF0512E51260F00908E87588
:1094AA00F0B484A8F08882E060ECF5D3B9000280B9
:1094BA00D5B9230050D0C395D292D15002F40409F1
:1094CA00FEE4FFFCAD0112572B7401FA25D475F0A6
:1094DA00B484A8F0AC06AB07125612EB30E7010CC5
:1094EA00E5D22C30D1029C9C8882F00AEAB501DCD4
:1094FA00E512244C50012285D3D28512D4A81280B9
:10950A00939004001295CA8C068B051295CAE4FF43
:10951A00F512F5118C148B13C3ED9BF9EE9CFA40EE
:10952A0012E51199E5129A500A8C148B138A128942
:10953A00118F528F82E0F9C3ED99FDEE9400FEE59A
:10954A0082245A5002244C75F0B48485F082E0FAE1
:10955A002DFDEE3400FEEB9AFBEC9400FCE92BFBAC
:0E956A00EC3400FC0FBFB4B0E55224D3400235
:1095780024B4F552C3E51333FBE51433FCE511FEBF
:109588002BFBE512FF3CFC125780E9F89095DC9321
:10959800F511FDEBF513FFECF514FE7C0012571ED8
:1095A8008F44E89096DC93FAAB13AC14125649AF8B
:1095B80003AE04AD117C0012571EEF7002F552F590
:1095C80045227C007B007F5AE02BFBEC3400FC0535
:1095D80082DFF522B4B4B4B4B4B4B4B4B4B4B4B49B
:1095E800B4B4B4B4B4B4B3B3B3B3B3B3B3B3B3B33D
:1095F800B3B3B3B2B2B2B2B2B2B2B2B2B1B1B1B144
:10960800B1B1B1B0B0B0B0B0B0B0AFAFAFAFAFAE56
:10961800AEAEAEAEAEADADADADADACACACACACAB74
:10962800ABABABAAAAAAAAA9A9A9A9A9A8A8A8A89C
:10963800A7A7A7A7A6A6A6A5A5A5A5A4A4A4A4A3CD
:10964800A3A3A2A2A2A2A1A1A1A0A0A0A09F9F9F04
:109658009E9E9E9D9D9D9D9C9C9C9B9B9B9A9A9A41
:109668009999999998989897979796969695959580
:1096780094949493939392929291919191909090C3
:109688008F8F8F8E8E8E8D8D8D8C8C8C8B8B8B8A05
:109698008A8A89898988888887878786868685854A
:1096A800858484848383838282828181818080808F
:1096B8007F7F7F7E7E7E7E7D7D7D7C7C7C7B7B7BD1
:1096C8007A7A7A7979797878787777777676767515
:1096D80075757474000203050608090B0C0E101149
:1096E80013141617191A1C1D1F2122242527282A8E
:1096F8002B2D2E303133343637393A3C3D3F4042FA
:1097080043454648494B4C4E4F505253555658596D
:109718005A5C5D5F606163646667686A6B6C6E6FF4
:10972800707273747677787A7B7C7E7F808183848D
:10973800858688898A8B8D8E8F909192949596973D
:1097480098999B9C9D9E9FA0A1A2A4A5A6A7A8A905
:10975800AAABACADAEAFB0B1B2B3B4B5B6B7B8B9E9
:10976800BABBBCBDBEBFC0C0C1C2C3C4C5C6C7C7E3
:10977800C8C9CACBCCCCCDCECFD0D0D1D2D3D4D4FB
:10978800D5D6D7D7D8D9DADADBDCDCDDDEDEDFE028
:10979800E0E1E2E2E3E4E4E5E5E6E7E7E8E8E9EA70
:1097A800EAEBEBECECEDEEEEEFEFF0F0F1F1F2F2CC
:1097B800F3F3F4F4F4F5F5F6F6F7F7F8F8F8F9F941
:1097C800FAFAFAFBFBFBFCFCFDFDFDFEFEFEFEFFCC
:1097D800FFFFFFFFC251E4F544F814FB900400A911
:1097E800007C0FC2D11298F7E82405F8B8B4F08BC2
:1097F80013E5122403FA244C5001FABBFF01227529
:10980800112C8A1912992E8F16203D12AA1975113A
:109818002312992E8F15751600303DE280117511AF
:10982800231298D6751500303D05E82F13F51575E8
:1098380011121298D6751400303D05E82F13F5144F
:10984800EA2404F552244C5002F552E4F51AF51BAB
:10985800F51CE516600AFB7A00AF137EFF12989C90
:10986800E515600AFB7A4FAF137EFF12989CE51648
:10987800600DFB7A00E5146006FF7ECF12989CAE5F
:059888001CAF1B7C0079
:10988D00AD1A12571E8F45EF2513F544D25122EF15
:10989D00F5F0A4FCADF0EBF5F0A49CFCE5F09DFD1E
:1098AD00EB8AF0A4FAABF0EF8EF0A49AF8E5F09BFA
:1098BD00F9E833F8E933F97B001257C4051AE51BB3
:1098CD002BF51BE4351CF51C22EA2511F9244C500F
:1098DD0001F9C2D11298F5303D428F00C3EA9511BE
:1098ED00F9500324B4F9D2D17C09E4FDFEFF89823D
:1098FD00E060062FFFE43EFE0D09B9B4027900DCED
:10990D00EDED20D118F51E24FE923D500F12572B70
:10991D00EFB503005006851E1FFB881222F51D8032
:10992D00E61298D6203D4374021299CD1298D62096
:10993D003D3874041299D51298D6203D2D74061217
:10994D0099CD1298D6203D2274081299D51298D629
:10995D00203D17740A1299CD1298D6203D0C740C27
:10996D001299D51298D6203D0122C3E89F605088E8
:10997D00148F158A1640081ABAFF0A7AB380060AA0
:0F998D00BAB4027A001298D6303D34C3E89FF97D
:10999C00602EC3E5149515FB6930E7D4E930E70375
:1099AC00F404F9EB30E702F404C3995002AA16E56B
:1099BC00142515C82F28FFE4FC33FE7D0412571E16
:1099CC00222AFA244C5001FA22C3CA9AFA500324D0
:0399DC00B4FA22B8
:10A62600C2B212C68FD2B275F83022C2B2F5F7C2E4
:10A63600B2C2B2D2B222D220D214740612A6317499
:10A64600C712A6311206FB12A659124089801F7442
:10A65600FF8001E4F5BCF5BDF5BEF5BF221206FB91
:10A6660085BF6C85BE6B756A0012A6D2C21FD2204A
:10A67600C2B275F705C2B2C2B2C2B2C2B275F705AE
:10A68600C2B2C2B2C2B2C2B2E5F7540170EFD2B2E0
:10A69600C22022D220C2B2F5F7C2B2C2B2856CF78E
:10A6A600C2B2C2B2856BF7C2B2C2B2856AF722D213
:10A6B60020C2B275F703C2B2C2B2856FF7C2B2C288
:10A6C600B2856EF7C2B2C2B2856DF722E56B70171E
:10A6D600E56A7013D22012A674740612A63174D8D5
:10A6E60012A699D2B2D21FC2202212A674D2207408
:10A6F6000612A631740212A6998FF7C2B2C2B2D25E
:10A70600B2C22022852E72E55F030354C0F8E55ECF
:10A71600543F28F57C30550122201F0612A6D23060
:10A726001F25D220C2B275F705C2B2C2B2C2B2C2EA
:10A73600B275F705C2B2C2B2C2B2C2B2E5F75401EF
:10A74600D2B2C220600122C21F12A9D512A674D2AB
:10A7560020740612A631740212A699787086F7083C
:10A76600B880FAD2B2C2207410256A54F0F56AE4B1
:10A77600356BF56BE4356C540FF56C22D380F0E540
:10A786004B75F010A4256A54F0F56AE5F080E1E512
:10A796006A24F054F0F56AE56B34FFF56BE56C342A
:10A7A600FF80D4E56A24FF80ECC380EBE56D24F0DE
:10A7B60054F0F56DE56E34FFF56EE56F34FF540F1A
:10A7C600F56F22D3E4356EF56EE4356F80F075A72C
:10A7D600047583048F827870E6F008B880FA75A74E
:10A7E600002275A7049004B47F20E4F0DFFD80EE1C
:10A7F60012A85012A87CC254C255E57F7002D255E9
:10A80600147002D254E54A30E00122B4061E2054E8
:10A816000F12A79512A92012A9B412A9EC02AAD167
:10A826001273D47E0412C687754A012220550F1270
:10A83600A76D12A99312A9D512A8F902AAA4127398
:10A84600D47E0412C687754A0522740312A6997827
:10A8560070E4F5F7C2B2C2B2A6F708B880F3D2B276
:10A86600C22022740312A699E4F5F7C2B2C2B2E579
:10A87600F7D2B2C22022E575F8541F30E40244E054
:10A88600F57585722EA2779226E57C543F30E50257
:06A8960044C0F55EE57C04
:10A89C0054C02323F55FE57F1414F55122856C6FAA
:10A8AC00856B6E856A6D22856F6C856E6B856D6AA6
:10A8BC0022E4FEFF740775A704F5838E8274FFF003
:10A8CC00DFFD75A7002274067E007FB012A8C2E4DB
:10A8DC00F55AF55B2275A704758306E55A600A756F
:10A8EC00F00A84E5F07002740AC4F58222307720F5
:10A8FC00E55A24024002055A12A8E1E55AF0E57324
:10A90C00F0E574F0E575F0E576F0E577F0E578F0D4
:10A91C0075A700223077F912A8E17F1074FFF0DFE1
:10A92C00FDE55A24F5500312A94B155AE55AB4FF0C
:10A93C0002055AC3E55A955B50D6755B0080D1125F
:10A94C00A8A97F0A056D056D12A6B5E4F5F7C2B28C
:10A95C00C2B2E5F7D2B2C22030E704DF02800512A2
:10A96C00A7B280E0056D12A6B512A8E1E55A24F64F
:10A97C00F07F06E4F5F7C2B2C2B2E5F7F0DFF4D22D
:10A98C00B2C22075A70022053FE53FB43C17753FC6
:10A99C0000053EE53EB43C0D753E00053DE53DB47D
:10A9AC001803753D00023CB8153FE53FB4FF177521
:10A9BC003F3B153EE53EB4FF0D753E3B153DE53D79
:03A9CC00B4FF03D2
:10A9CF00753D17023CB80542E542B43C0F75420095
:10A9DF000541E541B43C057541000540221542E5AE
:10A9EF0042B4FF0F75423B1541E541B4FF05754178
:10A9FF003B154022AC40AB41A842EC75F03CA42B78
:10AA0F00FBE435F0FC7A3C125612EB28FBE43CFCDD
:10AA1F0022AC3DAB3EA83F80E178AE8604AB3EE56D
:10AA2F003FC313F880111206F1ACBF53041FE5BEEC
:10AA3F0075F005A4FB7800EC75F03CA42BFBE43516
:10AA4F00F0FC7A1E125612EB28FBE43CFC2212AAF1
:10AA5F0035AE04AD0312AA28C3ED9BFBEE9CFC920E
:10AA6F004E4B700820110575367DD22E7A02125684
:10AA7F001275A7009004EEECF0A3EBF022E54D0465
:10AA8F0075F03C84E5F0653F600312A70A853F4DE2
:10AA9F002220740122C3E5709557FF24FD5021EF4A
:10AAAF0024EB400A78BD06B6001618068012EF2474
:10AABF0002400DEF2414500878BB06B600021806AA
:0AAACF00802BC3E5709557FF24FDAE
:10AAD9005021EF24EB400A78BB16B6FF16181680F2
:10AAE90012EF2402400DEF2414500878BD16B6FF6A
:07AAF90002181685705722B8
:10C6740012C67D12C67D12C67D7E0480067E0280AF
:10C68400027E017F0080087F6480027F017E00EFCC
:10C694004E6012E4FD0D1D0DEDC394AD40F7EF1F88
:06C6A40070ED1E80EA2289
:10C75100F5D8D2DCE5F520E7FBE5DA540FFEAFD9D9
:04C7610075D8002265
:10C40F007F767E06908A0F1265E2740412C7517C04
:10C41F00007D5212571EEFF875F00A84C0F07F7638
:10C42F007E2312BC727E29742E12BC857E2ED0E024
:10C43F0012BC727E35745612BC857F6B7E1190C410
:10C44F007812BCB3E824E04001220423F824E7501B
:10C45F0002781812C468D8FB227F6CE82411FE7989
:10C46F000512C6AA0E0FD9F922071DFFFFFFE080A4
:10C47F00000020C0000038E0000008F0000038F88D
:07C48F00000020FFFFFFE0A9
:10C4960012C4BE30E6022409540F75F00AA4F5153D
:10C4A60012C4BE30E6022409540F25152212C4BE5A
:10C4B600540F2275F000800875F044800375F0076C
:10C4C600E4206D07D5E0FAD5F0F722C2ACE54F625D
:10C4D6003885504F8599509247A26E926DA26F9201
:10C4E6006EC26FA247D2AC2212C4F8C4FA12C4F8C4
:10C4F6002A2212C4BE20E603540F2254072409221E
:10C2EB00E612C2F218E608FAC412C2F8EA540F4476
:10C2FB0030F924C6E950112407800D75F00A84C06B
:10C30B00F012C311D0E0443030530975F00085E0D2
:10C31B00E0D5F0FA3099FDC299F599623822E538EB
:10C32B0080F2E53812C2F2800812C313E53812C34B
:10C33B0013740D12C313740A80CE744012C313749A
:10C34B004080C5742C80C1742E80BD12C36EE9125F
:10C35B00C31F800312C36EE812C31FE53812C31F3D
:10C36B00023A80123A808003123A98744075380072
:02C37B008096AA
:10C7770085A0835383FE438380858384F07584007B
:01C78700228F
:10C0590074A212C77774A112C77774A612C777742E
:10C06900A412C77774C012C777742512C77712C094
:10C07900E975C70375C6FC75B90112A11A740812CE
:10C08900C751EE75F020A4FEEF54F80303032E24E4
:10C0990092C313FE24EA50027E16EE90C0D2932575
:10C0A900BCFE24E6501F24E8401B748112C777EEBA
:10C0B90012C77712C0F6744012C777742F12C77768
:10C0C90074AF02C7777E2680E1F7F7F8F8F9FAFB33
:10C0D900FCFDFEFF00000000010102020203030350
:10C0E900A8BCA9BDAABEABBFACC7ADC62288BC89D6
:0AC0F900BD8ABE8BBF8CC78DC62226
:10C5AF00D21AC006C007C0E075A7019000007EB781
:10C5BF0075A700EE12C777741012C777740412C7ED
:10C5CF007785A08343838185838475A7517F80E01E
:10C5DF00F0DFFC1EBEAFD9E4F5A7F584D0E0D0079D
:05C5EF00D006C21A2273
:10C7650075A711900000E4C583F0C58330E2F8F5A4
:02C77500A722F9
:10C6AA00EF20E723EE20E71F20E61C05A7C454036A
:10C6BA00F583EE5408C42FF582EE5407240983F556
:10C6CA00F0E045F0F005A72280402010080402019E
:10C6DA00EF20E723EE20E71F20E61C05A7C454033A
:10C6EA00F583EE5408C42FF582EE5407240983F526
:10C6FA00F0E055F0F005A7227FBFDFEFF7FBFDFE64
:10BC3200FDA42582F582E5F03583F583ED2290623D
:10BC42003D7A0475F00512BC327D0580607A05806C
:10BC5200027A04547FC0E0C083C082C394205001A2
:10BC6200E49061ED12BC4580309063467A05800510
:10BC72009063FC7A0675F00712BC327D07802E7A3B
:10BC82000580027A06547FC0E0C083C082C394203C
:10BC92005001E490638C12BC77D082D083D0E02232
:10BCA20090616B75F00A12BC327D0A7A07C2D180AC
:10BCB20002D2D1C0A7C082C083C007C006C0E03094
:10BCC200D10975A704E493FDE493FAEEFB75A7048A
:10BCD200EBFEEAFC7901D9067908E493F5D4E5D4C0
:10BCE20023F5D420E01612C6DA0EDCEA0FDDE1D02D
:10BCF200E0D006D007D083D082D0A72212C6AA8075
:10BD0200E89060AB75F00E12BC327D0E7A0812BC60
:10BD1200AF90615375F00212BC32E493FDE4A39339
:10BD2200FACE2408CE7C0812BD307C06AD02ED238B
:10BD3200FD20E00712C6DA0FDCF42212C6AA80F751
:10BB1D00F5D2C2D58036F5D2D2D58030F5D224F605
:10BB2D0050090E0E24A650030E0E0EE5D2F5D27559
:10BB3D00F0648485F0D3C2D57009D2D5742012BCBF
:10BB4D0085800312BC72CE2406CEE5D375F00A842F
:10BB5D0085F0D3700A30D507742012BC858003128E
:10BB6D00BC72CE2406CEE5D312BC72E5D222F5D23C
:10BB7D0075F0648485F0D3C2D58022F5D2C2D5800C
:10BB8D0025F5D2D2D5801FF5D275F0648485F0D31A
:10BB9D00C2D57009D2D5742012BC85800312BC6B3E
:10BBAD00CE2405CEE5D375F00A8485F0D3700A3026
:10BBBD00D507742012BC85800312BC6BCE2405CE34
:10BBCD00E5D312BC6BE5D222F5D2C2D58035F5D2C4
:10BBDD00D2D5802F30E70DF404C0E0742D12BC5384
:10BBED000E0ED0E0F5D275F0648485F0D3C2D57019
:10BBFD0009D2D5742012BC53800312BC40CE24044C
:10BC0D00CEE5D375F00A8485F0D3700A30D507746C
:10BC1D002012BC53800312BC40CE2404CEE5D312B7
:05BC2D00BC40E5D2223D
:1065CA007E008014D23C8002C23C7405FEF51EE4B3
:1065DA00FFF51DF51F203C3375A700E493700122D7
:1065EA00A3B40204051D8003B4010A051FEF2409A0
:1065FA00FFAE1E80E612BC857D06B440027D03B460
:10660A0021027D02EE2DFE80D27E0075A700E49362
:10661A00700122A3B40204051D8003B4010F051FF3
:10662A00EF2407FFAE1E80E612BC4F8008B45B0061
:10663A0050F612BC530EB4210280D30EB44002802D
:10664A00CDB42C0280C80E0EB45F0280C1B45B00C8
:10665A0040BC0E0E80B8E60812BC85EE2406FED5B4
:10666A0013F422908A14307409908A1830730390B4
:10667A008A1D0265E275F019D5E0FDD5F0FA123AE5
:10668A004612C345744F12C378744B12C334C322E3
:10669A00754B001266DD123A46D2AC12C4B9C5F087
:1066AA006024C5F0B440F412C4BEB4400312C4BEA0
:1066BA00B44F1C12C4BEB44B1612C4BE12C4BE12CE
:1066CA00C4BEC2ACC32212C4B9C5F070D5054BC250
:1066DA00ACD32230530975F008D5E0FDD5F0FA2283
:1066EA007F0375F019D5E0FDD5F0FA123A4612C3C8
:1066FA0045745712C378745012C313748112C313AA
:02670A00E56345
:10670C0012C313E56212C31378D0E612C31308B890
:10671C00D7F8E6F8795F30E702792FE912C3131244
:10672C00C31312C31312C313745812C3137443123A
:10673C00C313E412C313E8C2E775F00A84C425F04E
:10674C0012C3137864E612C31308B869F8E612C3CF
:10675C003412669A400122DF02800775F0008083B4
:10676C00D250C2ACD3221266DDC250123A46D2AC21
:10677C002002EF12C4B9C5F060E6C5F0B440F112C6
:10678C00C4BEB4400312C4BEB457D7F53812C4BE4D
:10679C00B450CF12C4BE12C4BEF56312C4BEF562AF
:1067AC0078D012C4BEF924A0500353015FE924E051
:1067BC004002795FA60108B8D8E8780612C4BED8A2
:1067CC00FB12C4BEFC53040FC4540F75F00AA42C66
:1067DC00FC249C50027C0078D78601E4B92F02D2AD
:1067EC00E72CF6786412C4BEF608B86AF812C4BE78
:1067FC00E538600302676E12C4BE12C4BEC2ACC3DD
:10680C0022908F1C8003908C7F7F2012661312C500
:10681C00AF02C685753400C26B1268D812C68512D9
:10682C006C50E516600312683802023B126EB4120B
:10683C00133712C5AF10002010010280F8126CBB88
:10684C00501312134212680D10000D10010280F843
:03685C001212E431
:10685F0080D7126A3C22C26BD22775480A122004D5
:10686F00753400126D8A753703C26A1228E5106AF3
:10687F000512022C80EA12022C126BE2126D3A12F0
:10688F006D96126EB412133712C5AF100038100187
:10689F000280F8126CBB501BE96515601812134289
:1068AF0012680D12C67D10001D10010280F8121221
:1068BF00E480C3D26B126D667516078559171220C7
:1068CF007D753500809A02023B126C501268FA12E5
:1068DF006D967F19126914908F497E121266157E7C
:1068EF0023E51602BBF190902580EF7862E41269E0
:1068FF000B78D0745F12690B18E4F6227F08F60844
:10690F00DFFC227F7B7E007810742012BC53CE24D4
:10691F0004FED8F5227F197E081266157E28908C0A
:10692F006B305303908C70026615C26B1268FA12AB
:10693F00694402023BC251126D96908F4112692435
:10694F0012130A126C507F201268E312C5AFE516BE
:10695F00700512C67A803675A6FF3051031266880D
:10696F00123A46D2AC200025306DFA126775400CF2
:10697F00126CBB4011126A3CD25180BB10500312F3
:10698F006812C25180D1D25112680D80CAC2AC2296
:10699F00D22775480A122004753400C26B126D8A13
:1069AF00753703C26A1228E5106A0512022C80E8B7
:1069BF0012022C126BE2126D3A126D961269D350BD
:0169CF00D7F0
:1069D00002023B908C7A12692412131C12C5AFC3B9
:1069E00010001310010510020E80F41266EA400137
:1069F0002212681280DDD3C2AC22D227C26B754846
:106A00000A122004753400126D8A753703C26A12A7
:106A100028E5106A0512022C80EAD26B126BE21292
:106A20006D3A126C0A75B901E5BCB2E7F5BC1240CB
:106A30008975160785591712207D80C8D26B126D93
:106A400066126C21E51775F01084240AF54824E8D5
:106A5000500375480A12201085585922D2207532E9
:106A60000012A8BD75A704900700751500126C0AE6
:106A700075B901E5BC20E705E515F0801004600D4F
:106A80006482600975BCFF75B90575B9020515E525
:106A900015242050D8E58224FE4003026B37A882DB
:106AA000187F0075A7007583078882E0FE75F004E3
:106AB000A4126BB5A9BCAABDABBEACBF1582E0FDEC
:106AC00075F004A4126BB5C3E995BC404C7052EA52
:106AD00095BD4045704BEB95BE403E7044EC95BF74
:106AE0004037703DEE75F004A404126BB5A9BCAA42
:106AF000BDABBEACBFED75F004A404126BB5C3E929
:106B000095BC4015701BEA95BD400E7014EB95BE08
:046B10004007700DBD
:106B1400EC95BF5008EEF00582EDF01582E5826039
:106B240009C3EF95825003026AAB0FC3E89F400389
:106B3400026AA375A70490070075C70375C6A8E089
:106B4400F5BCE0F5BDE0F5BEE0F5BF75B90575B976
:106B54000205C6E58224204006E5C6242050E0084C
:106B640075C70375C68075B901E5BC126B9FF5BC8A
:106B7400E5BD126B9FF5BDE5BE126B9FF5BEE5BF8B
:106B8400126B9FF5BF75B90205C6E5C6245850D6E9
:106B9400E5320470FB75A700C22022B4FF0122F97C
:106BA40075A704900700E582686005E06970F7E95D
:106BB40022F5C685F0C775B901E5BC645F7003753D
:106BC400BC27E5BD645F700375BD27E5BE645F70D7
:106BD4000375BE27E5BF645F700375BF272275C7C1
:106BE40003E54875F004A42480F5C6E55975F0045E
:106BF40084A8F00825C6F5C675B901A9BCAABDAB21
:106C0400BEACBF861522E515242050037515DFE5BB
:106C14001575F004A454FCF5C685F0C722E51724C5
:106C2400204028E51775F00484A8F00824A8F5C6C8
:0E6C340075C70375B901A9BCAABDABBEACBF44
:106C4200A61589BC8ABD8BBE8CBF12408922E4F591
:106C520016F51579FF126C0A75B901E5BCB4FF048B
:106C62000516A9150515E515242050E9891579FFA2
:106C720075C70375C6A875B90109E5BC04601B098F
:106C8200E5BD04601509E5BE04600F09E5BF0460B7
:106C92000905C6E5C6242050DD09891722751600AC
:106CA200751501126C0A75B901E5BC20E7020516DB
:106CB2000515E515242050EB227900E975F004A4AE
:106CC20054FCF5C685F0C775B901E5BC20E73078FC
:106CD200D066702B08E5BD66702508E5BE66701F9C
:106CE20008E5BF66701905C675B90108E5BC66708E
:106CF2000E08E5BD66700808E5BE667002D322097B
:106D0200E9242050B6C322126D29126D11A8017F09
:106D120008E0F608DFFB22126D29126D21A8017F1F
:106D220008E6F008DFFB2278D0796275A704758344
:106D320007EBC454F0F58222126C0A78D0126D541B
:106D4200E5BCF9C23C20E702D23C126D54786212D3
:0A6D52006D5475B901A6BC08A6BD7A
:106D5C0008A6BE08A6BF0805C622D220126C0A7867
:106D6C00D0126D78126D787862126D7886BC0886B8
:106D7C00BD0886BE0886BF0812408905C622125C73
:106D8C00A012C76512750202C5AF12C7657F007EDF
:106D9C0009908F2E1265E27F0A7E12E5150412BB54
:106DAC00297F1412B4681212E47F277E087513072A
:106DBC0078D0126660E6793E30E702792F7E34E9AE
:106DCC0012BC857F3D7E0190904112661520311BCF
:106DDC00303003127F39C23B127046126DFCD23B2D
:106DEC00127046126E0E12708D807C12AB0080E613
:106DFC00C23B7F447453201702744E7E0012BC8534
:106E0C008017D23B7F4F745720170274457E0012B7
:106E1C00BC857E06E51E12BC727E0CE51D12BC7292
:106E2C007E12E51C12BC727E17746412BC857E1C2B
:106E3C00E51B12BC727E22E51A12BC727E28742EDF
:106E4C00302602742712BC857E2DE51912BC727E89
:106E5C0033E51812BC727E39302607742C12BC81B3
:106E6C007E3BE53702BC72742D201702742B7F70A9
:106E7C007E1512BC85126E917E3A12BAD27E0190AA
:106E8C0090660265E27E1BE51C12BC727E21E51B3E
:106E9C0012BC727E27E51A12BC727E2DE51912BC4B
:0B6EAC00727E33E51802BC72126F32D8
:106EB700126F5D127234126D9612728C20171E10AB
:106EC700021B123B0D12B295126F1A1212EF7F348A
:106ED7007E2F12666D126DCF12C5AF80E21212E4DB
:106EE700203026203128C23B127046126F72786616
:106EF700127146D23B127046126F8778691271463B
:106F070012708D1270010271E912800280F212ABC9
:106F17001580EDE57D75F01084AAF075F00AA42AB6
:106F2700547FFA78D7E654802AF6227F277E08799D
:106F3700D08700C001D224B9D002C224127313D063
:106F470001A70010230909EE2406FEB9D7E3221989
:106F5700EE24FAFE80DB7E3479D7E7A2E792171298
:106F670072C079D7E7A21792E7F722C224C23B750E
:106F77001E007F447E001272D0801E1023ED802AEF
:106F8700D23BC2247F4F7E001272D8D2247E06E500
:106F97001E127305F51E1023E7D2247E0CE51D1281
:106FA7007305F51D303BD41023E1D2247E12E51C76
:106FB700127305F51C1023E17E1CE51B127305F502
:106FC7001B1023E67E22E51A127305F51A1023E833
:106FD7007E2DE519127305F5191023E87E33E518A0
:106FE700127305F5181023E87E393026027E3BE53B
:106FF70037127305F5371023E3227F707E1512725F
:01700700C8C0
:10700800C2247E1BE51C127305F51CD2247E21E5E3
:107018001B127305F51B1023E77E27E51A1273056B
:10702800F51A1023E67E2DE519127305F5191023BC
:10703800E87E33E518127305F5181023E82278D78F
:10704800E6C2E775F00A847866F537303B0578695B
:1070580085F0371270B630262BE53775F003A40497
:107068000475F00584FBE51975F00AA4251875F078
:1070780006A42BFBE435F0FC125834F537125834CB
:10708800F5188B1922E563FC339217AB6250031293
:1070980058A5305C0A7AD212562078401257C2AEF0
:1070A80004AF037C277D1012572B8F1C8037E6FD19
:1070B80033921718860418860350031258AD7A09BC
:1070C800792778C01257BF8B1EADD3ACD2AB0679E7
:1070D800EA78601257BD8B1DAF06AED27C177D7063
:1070E80012572B8F1CAF05AE047C037DE812572B7B
:1070F8008F1BAF05AE047C007D6412572B8F1AEDF1
:1071080075F00A84F51985F01822EC3392175003AC
:107118001258A5751D30301786751D2D808178424F
:107128007B607CEA800678407B207C4E12ABE0795D
:087138002778101257BD8B1CD3
:10714000AF06AED280AB30262AE51975F00AA42529
:107150001875F00AA42537FBE435F0FC7A051256C1
:10716000128C068B077C007D0312571E8E048F0342
:10717000127080E51E75F00AA4251D75F00AA4257D
:107180001C75F006A4251BFBE435F0FC7A0A1256A8
:1071900012EB251AFBE43CFC7A0A125620EB251967
:1071A000FBE43CFCE43DFD7A0A125632EB2518FB69
:1071B000E43CFCE43DFD3017031258ADA60518A6CB
:1071C0000418A60378D7E6A2E7923DC2E775F00A55
:1071D00084FCABF0303B0EAB37EC75F00AA42BA26D
:1071E0003D92E7F622AC3780F0127204305C0A7AE6
:1071F0004012562078D21257C23017031258A58C6D
:10720000638B62221272147A0A125612EB2518FB53
:10721000E43CFC22E51C75F00AA4251B75F00AA4C9
:10722000251AFBE435F0FC7A0A125612EB2519FBFD
:10723000E43CFC2212726612C681C202C2231272A0
:107240006610000810010510021B80F51031ED10CA
:05725000300D102604C2
:10725500D22680E3D230C23180DDD231C23080D730
:10726500227F3590902A12661390904820300F9017
:10727500905E2031099090392026039090311F7E31
:10728500171265E202C5AF7F357E01908C4A126602
:10729500157F347E3A1273B5744E12BC8512C5AF94
:1072A50012C681C2027F347E3AD217751159751202
:1072B5004E802675112E751227801E75113E75128A
:1072C5002F801675112B75122D800E75114E7512A6
:1072D5005380067511457512571273B5E5113017B0
:1072E50002E51212BC8512C5AF1000081001051089
:1072F500020B80F5D23C1017E3D21780DF0273B082
:107305004430F812730FE8540F22C2218002D221B3
:10731500A224922292231273B5E830E709D23C7475
:1073250030302102745FF812BC8512C5AF100034ED
:1073350010010510025D80F5D23C1022661023670E
:10734500B43909745F2021DF743080DBB45F0474C5
:107355002D80D4B42D04744180CDB45A047430808A
:10736500C60480C3D23C302406102237102338B41B
:107375004104742D80B1B42D04745F80AAB45F04F8
:10738500743980A3B43009745A20219B74398097CD
:10739500148094B47108D223E812BC85800DF8C21C
:1073A50023800874718001E802732C9073CA8003EE
:0373B5009073C60C
:1073B800C007EF2408FF12BCB3D00702C5AF02050F
:0673C800F8F802050000C8
:10C5060075A70090C53875F02D84C2D5C2D16017C5
:10C51600D2D1146007D2D514600DC2D1E5F093FCD8
:10C52600742D95F093FB22E5F093FB742D95F09313
:10C53600FC220009121B242C353E474F58606870B8
:10C546007880888F969DA4ABB2B8BEC4CACFD4D922
:10C55600DEE2E6EAEDF0F3F6F8FAFCFDFEFFFFFF99
:10C5F400D23D8002C23DED8BF0A430E70205F0C3CA
:10C60400E895F020D50425F025F0FEED8CF0A4305B
:10C61400E70205F0C3E995F030D10425F025F0FFD9
:10C62400203D0B2487500122EF24CC40012202C676
:01C63400AA5B
:10C10300203A437E1C7F5312C6AA7F5912C6AA1E29
:10C113007F5712C6AA7F5512C6AA7E2312C6AA7FCC
:10C123005712C6AA1E7F5912C6AA7F5312C6AA1F48
:10C133007E2012C6AA7F5A12C6AA7E1E12C6AA7FE4
:10C143005212C6AA800A7E1C7F5390C19612BCB3BA
:10C15300200C0A303A077E1F7F4102B4C430741C9E
:10C16300E5716018E57012C506781F79567D0912CE
:10C17300C5F8303A0312C1800DBD16F322C0060E76
:10C1830030D5021E1E12C6AAD0061F30D1020F0FD1
:10C1930002C6AA070700386C446C380005052070F6
:0AC1A300D8702005057088A8887088
:10B2BA0030122D9090707F717E2F12661512A8A9F8
:10B2CA007A0AC23D12B52C203D16DAF812B42E7C49
:10B2DA00007D0312571EEFA2D17E237F6512BD4A5D
:10B2EA00227F567E0512B4747F3D12B4877F6F1297
:10B2FA00B4877E1F7F4112B4C47E0A7F4112B4E62E
:10B30A007E227F5912B4E62012012212A8A9857A58
:10B31A001D855E1C857B1B855F1A7AC0C23D12B5EE
:10B32A002CBAB7048C1C8D1D203D5212B42E7C0001
:10B33A007D1412571E74562F20D1029F9FFF24CBD3
:10B34A0040028037EF248850028030EA1475F003F7
:10B35A0084FE12C6AAC3E51B957BFEE51A955F9289
:10B36A00D55004EEF404FEEEC313FE24E0400C7440
:10B37A001F2E30D5029E9EFE12C6AADAA120120105
:10B38A00227F5212B4247F5A12B4247516007517FC
:10B39A0053801E201201227F157E2D742012BC8537
:10B3AA007E2D7F1C12C6DA0EBE40F975162F751750
:10B3BA0015AC1CAD1D12B42E7C007D0312571EEF76
:10B3CA00A2D1AE16AF1792D175F080305C04F5F0B9
:10B3DA008001A4A2E792D5E5F075F03284F8E5F091
:08B3EA0075F00584C0E0E5F0F8
:10B3F200A2D533C0E0E8601E12BC6BEE2406FED07C
:10B40200E0F8D0E012BC6BEE2405FE742C12BC8571
:10B412000E0EE802BC6B742B20D102742D12BC8577
:10B4220080D97E1112C6DADEFB02C6DAC3ED957A46
:10B43200FFEC955EFE92D150031258952212A8A9F4
:10B44200857A1D855E1C7A0AC23D12B52C203D0606
:10B45200DAF88C1C8D1D227F1512B4607F327E3E7D
:10B4620012C6AADEFB227E0E12C6AA0EBE31F92237
:10B472007E0112C6AA0E0EBE3FF8227E3312C6AA63
:10B482000EBE40F9227E047D1112C6AA0E0E0EDDFA
:10B49200F81F1F7E35909074305C057E3190907855
:10B4A2000266157405305C097E32740112BC407468
:10B4B200067E3612BC407E3A740012BC407E3D02CB
:10B4C200BC407D0F12C6AA0F0F0FDDF8227F737DDD
:10B4D2000380047F727D0512C6AA0FDDFA227F71F6
:10B4E2007D0780F37D0A12C6AA0E0E0F0FDDF7222A
:10B4F200203D0712306F7003D23D22056D12A6B5B2
:10B50200E4F5F7C2B2C2B2ABF7F5F7C2B2C2B2E526
:06B51200F7FA30E411EB32
:10B51800251DF51DE4351CF51C0519EA30E3010E5F
:10B52800D2B280117803203D0712306F7003D23DEC
:10B5380022D8F3056DE56D2409F56D12A6B5E4F57D
:10B54800F7C2B2C2B2ADF7F5F7C2B2C2B285F71B05
:10B55800F5F7C2B2C2B2E5F7FCD2B2C220543F300E
:10B56800E50244C0CC54C02323F51AE56D24F6F552
:02B578006D2242
:10C37D007E017F0990C3FB12BCB32051097E037F60
:10C38D0000743F02BC85E4FEFFC3E54512B80BFD0A
:10C39D00940AED403D9464ED4002746312BB237E1C
:10C3AD00017F09E552240575F02D84AAF075F0057D
:10C3BD00A4CA75F00B842A90C3E69312C506BCB8C7
:10C3CD00027BB87D04EE2DF8EF2DF90D12C5F4DDCD
:10C3DD00FB227E0312BC7280C6000C1622222D3960
:10C3ED00444F4F5A66707C7C87939EA9A90009091A
:10C3FD00080041000000000088800000000041009E
:02C40D00080025
:10B80B00305D0A75F08AA42480E5F03400227F00B5
:10B81B002074147E110F90B8A512BCB37F0A7E0A58
:10B82B00E52E540702BB3A7E0BE571B4FF2DE551B3
:10B83B0024025003755100E55112B80B75F005A4A5
:10B84B00ACF0FB1255E87E0D781CE66004E612BCEA
:10B85B006BEE2405FE18B818F4800612B80B12BB59
:10B86B00297F0C7E11E571602B0EE57064B46024AA
:10B87B0064B475F03284C0F012BC6BCE2405CED00C
:10B88B00E075F00584C0F012BC6BCE2405CED0E081
:10B89B002302BC6B90769B0265E2070FFFFF9EE7CE
:10B8AB00AD6B9C6BAD6B9D67FFFF75548030745D0A
:10B8BB0078BD79BBE6FC27FB1819E6FD37F9EBF8E9
:10B8CB007B001257C48B547F087E11A80690B919C0
:10B8DB0012BCB330100F20730C7F0A7E1712C6DA1E
:10B8EB000E0E12C6DAE5542483E554500224FA7581
:10B8FB00F01984FB90B9219328FEEB90B92B93FDA3
:10B90B0012C6AA0F0F12C6AA1F1F0EDDF322030FBA
:10B91B000100FFFE03800000000007070D0C0B0A5F
:10B92B0005040302010102030405E57E7001227F79
:10B93B00357E00746F12BC857E06E57E12B80B0255
:10B94B00BB94202C012290B95702BCB3050EFFF01B
:0CB95B00E01CF004F81CFFF03012012288
:10B967007F6E7E00908A2F12BCB37F1512B4607F62
:10B977001F12B4607F2912B4607F177E06E53F303F
:10B98700E00B909088305C0390909C8013207407A4
:10B997007E01908A4F800990907D305D0390909250
:10B9A7001265E2307306E54E6002154E205718E522
:10B9B7004EB401131206F1C3E55C9560F5BCE55D75
:10B9C7009561F5BD1240897F217E01E53F30E02179
:10B9D700305705908B148016E54E7005908B2080AC
:10B9E7000D908A5B1265E27E30E54E02BB8E1265D2
:02B9F700E2224A
:10B9F9001255BA7F207E05751900781DC2D5E6302B
:10BA0900D51712BC6BEE2405FE18B818F17E1F7409
:10BA190063305C02746502BC857005B8191880E250
:10BA2900D2D5CE24FACE746B301702742D12BC8590
:10BA3900EE2406FE80C8742012BC8180C87F007E77
:10BA490023AC5EAB7A1255BA781DC2D5E630D50C57
:10BA590012BC72EE2406FE18B818F1227005B81946
:10BA69001680EDD2D53017E4CE24FACE742D12BC4F
:10BA790085EE2406FE80D5742012BC8580D512552A
:10BA8900BA781DC2D5E630D51612BC40EE2404FEA4
:10BA990018B818F10E745E305C02742702BC4F703E
:10BAA90005B8191680E3D2D53017DACE24FCCE7446
:10BAB9002D12BC53EE2404FE80CB742012BC53809B
:10BAC900CBC23D12BADD0F0F0E0E7463305C0274E7
:10BAD9006502BC851255BA781DC2D5E630D50C125F
:10BAE900BCA2EE2408FE18B818F1227005B8191680
:10BAF90080EDD2D5301716740BCE24F8CE12BCA225
:10BB0900EE2408FE80D5740C12BCA280D5303DCB42
:04BB1900740A80E545
:10BEF0007F797E24E55F30E70122AC5F1CAB7B12CB
:10BF000055E8E51B700E742012BC85EE2405FE1268
:10BF1000BF3E800C12BF3EE51B12BC6BEE2405FE3B
:10BF2000E51A12BC6BEE2405FE742C12BC850E0EB5
:10BF3000E51912BC6BEE2405FE745E02BC85742DFF
:10BF4000201702742B12BC85EE2406FE22E55F301A
:10BF5000E70122AC5F1CAB7B1255E8E51B700E7449
:10BF60002012BC53EE2404FE12BF97800C12BF9720
:10BF7000E51B12BC40EE2404FEE51A12BC40EE2480
:10BF800004FE742C12BC530E0EE51912BC40EE24B4
:10BF900004FE742A02BC53742D201702742B12BCA9
:06BFA00053EE2404FE2212
:10BD42007E257F09A275E579C23D6002D23D92D17E
:10BD520075F080305C04F5F08001A4A2E792D5E58D
:10BD6200F075F03284F8E5F075F00584C0E0E5F096
:10BD7200A2D533C0E0E8602712BCA2EE2408FED0B0
:10BD8200E0F8D0E012BCA2EE2408FE0F0F205A1FEA
:10BD9200746012BC851F1FEE2404FEE802BCA2746C
:10BDA2000C303D06740A20D1010412BCA280CC20C2
:10BDB2005904742E80DC205804746180D57462802A
:10BDC200D1A275E579C23D6002D23D92D175F08073
:10BDD200305C04F5F08001A4A2E792D5E5F075F09D
:10BDE2003284F8E5F075F00584C0E0E5F0A2D533C1
:10BDF200C0E07F3E7E1CE8602012BD03D0E0F8D098
:10BE0200E07F3E7E2812BD037F447E32742E12BC38
:10BE1200857F3E7E37E802BD03303DE0740A20D1C3
:07BE2200010412BD0380D5ED
:10B57A00E54424F64001227800E5520475F003847C
:10B58A00F9E928FE24C45001FE12B5B212B5BE1E56
:10B59A0012C6AAC3E998FE5003243CFE12B5B21E95
:10B5AA0012C6AA08B81FDA22EE2420FE24C25003CB
:10B5BA002402FE22E824F1E8C2D55006D2D5E8F4E6
:10B5CA00241F23FF90B64093CF0493FAE545F5F084
:10B5DA00A4ACF0FB125649E544F5F0A49BFBE5F058
:10B5EA009CFCEB2420FBEC3400FC12B621FAE54566
:10B5FA008FF0A430E70205F0E5F020D502F4042A22
:10B60A0075F00520190375F00384FF24DF50027FCB
:10B61A0020C374329FFF22EC24F0500BEB2460EC21
:10B62A00340090B6909322EB33FBEC33FCEB33EC13
:10B63A003390B6609322FF00FF03FA0BF318EA2A4D
:10B64A00DE40CF58BE73AB8D96A880C068D64FE84F
:10B65A0035F51BFD00FF00080B0E10121415171804
:10B66A00191B1C1D1E1F20212223242526262728BC
:10B67A00292A2A2B2C2D2D2E2F2F303131323333DC
:10B68A00343435363637373839393A3A3B3B3C3C2D
:10B69A003D3D3E3E3F3F4042444648494B4D4E5059
:10B6AA005253555658595B5C5D5F606163646566C9
:10B6BA0068696A6B6D6E6F70717273747677787978
:10B6CA007A7B7C7D7E7F8081828384858687888958
:10B6DA008A8B8B8C8D8E8F9091929394949596975A
:10B6EA009899999A9B9C9D9E9E9FA0A1A2A2A3A471
:10B6FA00A5A6A6A7A8A9A9AAABACACADAEAFAFB098
:10B70A00B1B1B2B3B4B4B5B6B6B7B8B9B9BABBBBCE
:10B71A00BCBDBDBEBFBFC0C1C1C2C3C3C4C5C5C60F
:10B72A00C7C7C8C8C9CACACBCCCCCDCECECFCFD05A
:10B73A00D1D1D2D2D3D4D4D5D5D6D7D7D8D8D9DAAD
:10B74A00DADBDBDCDDDDDEDEDFDFE0E1E1E2E2E306
:10B75A00E3E4E5E5E6E6E7E7E8E8E9EAEAEBEBEC65
:10B76A00ECEDEDEEEEEFEFF0F1F1F2F2F3F3F4F4CB
:10B77A00F5F5F6F6F7F7F8F8F9F9FAFAFBFBFCFC37
:10B78A00FDFDFEFEFFFFE54524FD400122E55204D2
:10B79A0075F00384241FFE24C250032402FE12B74C
:0DB7AA00E1EEFD241EFE24C250032402FE29
:10B7B70012B7E1E544240275F00520190375F0037B
:10B7C70084F4042432FF24EE500F12B7D6AE051EC0
:10B7D7001E7C0512C6AA0EDCFA227F1512C6AA0F16
:10B7E7000FBF2DF822E5530475F00384241FFE24B0
:10B7F700C250032402FE12B8010E7F2312C6AA0FFD
:04B80700BF2DF92236
:10BE29007E397437301902745512BBDB802175A72E
:10BE3900007E007F2F90BECB12BCB3205DE27E64F2
:10BE49003019027EA09004C3E02E7E3512BBF1307A
:10BE5900745A301257E54AB4040122B4060122E5A6
:10BE69007112B60AEFFDE5700475F00384241EFE15
:10BE790024C2401F2403501E90BEB6600990BEBD67
:10BE890014600390BEC4E493A3B4FF0122FE12BE62
:10BE9900AA80F32402FE7C04EDFF12BEAA0EDCF890
:10BEA90022EDFF12C6AA0FEF24CE50F7223B3C3DEC
:10BEB9003E0001FF3C3D3E010203FF3E3F010203FC
:10BEC90004FF05387001100240078080011003400B
:10BED900040060015003C0070017FCA7FADFF43F14
:07BEE900E000A00240078009
:10C56600AF177E00E53C12BB1D7E0C742E12BC85F7
:10C576007E12E53B12BB1D7E1E742E12BC857E24E8
:10C58600E53A02BB1D7E0E78ADE612BB887E1874B6
:10C596002C12BC857E1B18E612BB887E25742C12D5
:09C5A600BC857E2818E602BB8862
:10C635007F797E16743B12BC817E18E53F12BB885C
:10C645007F797E0078AEE612BB887E0A743B12BC09
:10C65500817E0CE53E02BB887F797E00E54012BBFA
:0FC66500887E0A743B12BC817E0CE54102BB88C3
:10C1AD00787512C1FD7453201702744E207406E584
:10C1BD002E54074430AF1712C2277E3BE57DC45481
:10C1CD000F12BC722074077E07742012BC8578781C
:10C1DD0012C1FDE5172409FF74572017027445207D
:10C1ED007402742012C2277E3BE57D540F02BC728F
:10C1FD00E6FD33921718860418860330170312587C
:10C20D00AD791778701257BD8B13AF06AED27C0087
:10C21D007D6412572B8F148D15227E0012BC857EE6
:10C22D0007E51312BB3A7E19746412BC857E20E5B6
:10C23D001412BB1D7E2B742E2073030E742C12BC96
:08C24D00857E2FE51502BB1DE3
:10C25500C234E54A602E7A2420E00E7A2614146052
:10C26500087A28141460027A297F717E00EA12BCCC
:10C2750085205505205406800B745B8002745C7E16
:10C285000012BC8530262CC2269091D37F6812659A
:10C29500CA7F66A85AE54AB4060108E875F06484C1
:10C2A500740AC5F084C0F012BCA2EE2409FED0E0E9
:10C2B50012BCA2200811E537B402032041097F36DC
:10C2C5007E2E744112BC5322E54375F008A49535C2
:10C2D5005013E59020E20ED2347F6F122D640F903B
:06C2E5008AA01265E222AE
:10BFA60020144F740512C751EF33EE33F9EF030334
:10BFB600541FF5F090BFF9E993A4C5F013C5F0132B
:10BFC600C5F013C5F013C5F0135403FCE5F013FBDD
:10BFD600E9242093C9244093C39BC4540FFBE99CD6
:10BFE600C4FC540FF9EC54F02B2446F57BE934F6E7
:10BFF600F55F22FFFFFFFFFFE6C5AD9C8F857D77CE
:10C00600726E6C6A696A6A6C6F747A828D9DB4D935
:10C01600FFFFFFFAE9DCD3CEC9C6C3C0BEBBB9B7C2
:10C02600B5B4B2B0AFADABAAA8A6A4A2A09E9C9987
:10C0360096918C00381CE735D137246F00C5B3C103
:10C04600E61F66B60E68C21867AADBF4EDB9467538
:03C0560010A20035
:10C73100D2A27408D2A1D2A300C2A3C2A1D2A300E3
:10C74100C2A3D5E0EF7405D2A300C2A3D5E0F822BD
:10C70A00C2A3D2A2D2A1D2A300C2A375F0083392C7
:10C71A00A1D2A300C2A3D5F0F5C2A175F003D2A39A
:07C72A0000C2A3D5F0F822C4
:10AEE90012C70AD2A300C2A3C2A175F008E4D2A373
:10AEF90000C2A3A2A233D5F0F5FE75F008E4D2A3EF
:10AF090000C2A3A2A233D5F0F5FFD2A300C2A322A7
:10AF1900E478806608B88BFB70012274D512AEE91B
:10AF29007881C3EE13FEEF13F692D118EE2460F682
:10AF390074D612AEE97888EF33CE33CE33CE33CE22
:10AF490033A2D192E25407FCEEFB7A08125612ECB6
:10AF5900244FF608EBF674D912AEE9EF543F788224
:10AF6900F67886EF33CE33CE33CE33CE335403F671
:10AF790008EEF618161608E6C4FF54F0F618E6C4EB
:10AF8900CF540F2FF674DA12AEE9EF232354FC786D
:10AF990083F67884EEF608EF54C0F67880E4660804
:10AFA900B88AFBF62212AEF17889C3EF96FF18EE44
:08AFB90096FEA2E7921650106B
:10AFC100125895740FF8F912565FEF2CFFEE3DFE03
:10AFD100788BEEF608EFF622E6182016072CF7E636
:10AFE1003D19F722C39CF7E69D80F66A405E8056C4
:10AFF100E050F04B0044803DC0384031D02BA025BB
:10B00100601F2018D014000F000AA001440158014C
:10B01100680178018801A001B401D001EC0210029D
:10B0210038026802A002DA030C034D78BE80208545
:10B031008E8A9D8F4D95BA9A97A0BEA631AC53B218
:10B041002AB801BD6AC1EDC4D1C78812AEF1788DAD
:10B05100EEF608EFF67887798C12565F788379904F
:10B0610012AFD97885798C12565F7881799212AFB7
:10B07100D9788DE624E4FE08E63392D13392D55493
:10B08100FCFFEEA2D133A2D533FE780F799212568E
:10B091005F78947990C3EC97F61819ED97F6799447
:10B0A10090AFEC7F1F7D11EF93C3971F19EF93971B
:10B0B1001F091DED600240EF0F90B00C798DEF93E9
:10B0C100F7090FEF93F7788E799412565F90B02CB1
:10B0D100EF93C39BFB1FEF939C2420FC7897E62BF7
:10B0E100F618E63CF618E436F6740612C751D23764
:09B0F100EE24F74006240250028F
:10B0FA00C237EEFCEFFD740712C751C3ED9FFFEC98
:10B10A009EFE78B7E6FD337C0050011CEF2DFFEE62
:10B11A003CFE78D8E6C4540F2FFFE43EFE789CEF3D
:10B12A0026F618EE36F62220141220370F789DE6FE
:10B13A00B4050912B1E412B21912B25D22201459EF
:10B14A007897799A12B27812581DC3EE9420FE921B
:10B15A004550031258957C007D0512572B30450344
:10B16A0012589512C0E91206E7E5BC2FF560E5BD55
:10B17A003EF56120E71124F8500DFAC3E5609AF50F
:10B18A0060E5619400F5611206F1E5BC2560F57A87
:10B19A00E5BD3561F55E12C0F67897799AC3E697F0
:10B1AA00FB1819E697FC7A0212561230370B7A020C
:10B1BA00125612ECFEEBFF800312B1E412B2192010
:10B1CA00140312B25D78957998E6F776000809E6D5
:10B1DA00F776000809E6F7760022799CE77700FB04
:0BB1EA0019E77700FC789DE6B405062D
:10B1F500EB33FBEC33FCECA2E792D550031258A5D8
:10B205007A32125620ECFBEDFC30D5031258A5EC32
:10B21500FEEBFF22EE2408FE7404203711789DE62C
:10B22500B40504740C8007F42406C323540FFD7C75
:10B23500001255FE789FE6FC08E6FBC374109DFAE4
:10B24500125620EFF8EEF912581DE878A02FF6FFF8
:10B2550018EE39F62480FE2292754003125895EFB8
:10B2650033EE33F579C276307508E57924F150026D
:10B27500D27622E627FB1819E637FC1819E637FDC2
:10B285002212A8507F087871793A12B2A1023CB80F
:10B29500855E63857A62787379647F06E6F70809C7
:10B2A500DFFA227864797380F1787379AF80EB786F
:05B2B500AF797380E594
:10559800E4FEFFFC7D0A791DE7540F2FFFE43EFE71
:1055A800B919028006191255FE80ED3017031258FA
:1055B8009522305C2BEC33921750031258A5EC243B
:1055C800D950047C277B007AD2125620EB33CC3397
:1055D800CD33CC33ED33FBEC33FC3017031258A535
:1055E800EC33921750031258A57919125834F70959
:1055F800B91DF8A70322EFF88DF0A4FFEDC5F0CE92
:10560800A42EFEEC88F0A42EFE22EB8AF0A4FBE583
:10561800F0CC8AF0A42CFC22EB8AF0A4FBE5F0CCB9
:105628008AF0A42CFCE435F0FD22EB8AF0A4FBE51B
:10563800F0CC8AF0A42CFCE435F0CD8AF0A42DFD42
:1056480022EB8AF0A430E70205F0E5F0CC8AF0A45A
:105658002CFBE435F0FC2286F0E7FDA4FAABF01948
:06566800E786F0A42BFB15
:10566E00E435F0FC18E68DF0A42BFBEC35F0FCE4F1
:10567E0033FDE687F0A42CFCED35F0FD22EB89F02E
:10568E00A4CBAEF08AF0A42EFEE5F03400FDEC893A
:10569E00F0A42EFEE5F03DFDE433CC8AF0A42DFD02
:1056AE00E5F03CCEFC22EB89F0A4CBAFF08AF0A45F
:1056BE002FFFE5F03400FEEC89F0A42FFFE5F03E5D
:1056CE00FEE433CC8AF0A42EFEE5F03CFCED89F02E
:1056DE00A42EFEE5F03CFCE433CD8AF0A42CFCE5D0
:1056EE00F03D8E058C068F04FF22C2D5EC30E70507
:1056FE00B2D512589DEE30E70DB2D512589512570D
:10570E002B12589D800312572B30D5031258952219
:10571E00C3EC13C0E0ED132FFFD0E03EFEBC000B38
:10572E00BE0029EF8DF084FFADF022E4CCF975F0C8
:04573E0008EF2FFF42
:10574200EE33FEEC33FCEE9DEC994005FCEE9DFE43
:105752000FD5F0E9E4CEFD22EDF9F5F0EE8420D28A
:105762001CFEADF075F008EF2FFFED33FD400799F9
:105772005006D5F0F222C399FD0FD5F0EA22EC33A0
:10578200EE3400FEEF3400FF7D007A0079007809E4
:10579200C3ED9AFDEE9BFEEF9CFFB392D54009ED5F
:1057A2002AFDEE3BFEEF3CFFA2D5E933F9ED33FDD6
:1057B200EE33FEEF33FFD8D92279007A00C3801589
:1057C20079007A00C3EA13FFE913FEE8132BFBEE1C
:1057D2003CFCEF3DFDE4F5D2F5D333FE7F19C3EE79
:1057E20098FEE5D299F5D2E5D39AF5D3B392D54096
:1057F2000DEE28FEE5D239F5D2E5D33AF5D3A2D59E
:02580200EB3386
:10580400FBEC33FCED33FDDF0122EE33FEE5D23356
:10581400F5D2E5D333F5D380C3EDC454F0FEECC424
:10582400FF540F2EFEEF54F0FFEBC4540F2FFF2252
:10583400EC75F00A84FCEB54F025F0C475F00A848E
:10584400C4CBC454F025F0C475F00A842BFBE5F0F6
:1058540022AC10AB11125834A904AD03FA7C197BA5
:1058640099125612AE04AF03EA75F006A4F8AC120E
:10587400AB131258342875F00A8485F014F8EF2B12
:10588400FFEE3CFEEF28FFE43EFEE43DFDE439FC80
:1058940022C3E49FFFE49EFE22E4C39DFDE49CFC3E
:1058A40022C3E49BFBE49CFC22C3E49BFBE49CFC3E
:1058B400E49DFD2275D4107B807A0079807800EA1B
:0A58C400F5F0A4FCADF0EBF5F0A444
:1058CE00FEAFF0EB8AF0A4C333C5F033C5F092D52A
:1058DE002DFDC5F03EFEE430D501043FFFB5150D9C
:1058EE00EEB51409EDB51305ECB51201224006EA2A
:1058FE0098FAEB99FBD5D40ABB0001220ABA000133
:10590E000B22C3E913F9E813F8EA28FAEB39FB8006
:10591E00A478087B807D807C00EDF5F0A4FAE5F09C
:10592E008EF0B5F007EA8FF0B5F001224003ED9B43
:10593E00FDD827BDFF0122EDF5F0A4F9A8F0ED0486
:10594E00F5F0A4C399FAE5F09813CA1329F9E83AC9
:10595E00F8C3E99FE89E50010D22C3EB13FBED2B1C
:10596E00FD80B67473F8F9E627FB0809E637FC08E4
:10597E0009E637FD30E7031258ADEB33FBEC33FC91
:0B598E00ED3323FD242083F8ED241CE2
:1059990083FFED241883FAED241483F9EF99F9E8CC
:1059A9009AFA12568BEF9DFFE89EFE22FFFFFFB683
:1059B900FED7FD63FB5DF8C4F59BF1E3ED9EE8CFEF
:1059C900E379DD9ED743D06BC919C153B91CB079AE
:1059D900A7709E06943F8A237FB674FF6A045ECB44
:1059E900535B47BB3BF1300423FB17DE0BB2C21DEF
:1059F900C232752C00C3E5679576FBE5689577FC9F
:105A0900E5699578FD30E705D2611258AD24F0506B
:105A190003125ACBAA06A9071256B4EC2480E43D16
:105A2900FBF9F51AE43EFCFAF519E43F6002D232BB
:105A390012568B8B128C138D148E15C3E5649573D6
:105A4900FBE5659574FCE5669575FD30E705D26261
:105A59001258ADEBF9F51FECFAF51DED6002D232E3
:105A69003032012212568BEB2512F512EC3513F563
:105A790013ED3514F514EE3515F51540E10258B856
:105A89001259F720323BEB242E40D3EA2401CB34C0
:105A990000FC7A07793D12568BC010C0118E108D0B
:105AA900118C128B13E4FCFD7E077FD012A0978521
:105AB9001203851302D011D010BB0005BA0002D21F
:105AC9001D22B261C374809BFB74F59CFC74209DFC
:015AD900FDCF
:105ADA0022303F777F747E0112B4747E1F12B4E0C5
:105AEA0075A7009004EDE0A2E792171392E7FC1560
:105AFA0082E013FB3017031258A5BC004EEB604B33
:105B0A0020E74820E64510E513201707C3741F9BBA
:105B1A00FE80027E1F12B4D50EDBFA22FB20170983
:105B2A007E00C374209BFB8008EB241FFE74209B1D
:105B3A00FB12B4CF0EDBFA2275A700758307E5596D
:105B4A00C4440FF582E0A2E79252222212B2AE12A8
:105B5A005B42C2E775F00A84FEAFF075A704538270
:105B6A00F17864125BCAAE077867125BCA75A70040
:105B7A00E57DC4540FFEE57D540FFF7873125BBEBA
:105B8A00AE077876125BBE74AF125973125A891235
:105B9A0006E2A9BDE5597002A9BCE975F00AA4F9A3
:105BAA00EA999004ECF0A3EB95F0F0A2E7923DD2CB
:105BBA003F02B2B4860308860408860518188006D0
:105BCA00E0FBE0FCE0FD7A0A12563220E70CEB2EED
:0D5BDA00F608E43CF608E43DF622C3EB9E1D
:105BE700F608EC9400F608ED9400F622C23F302A3E
:105BF7000F78A87600223038FCC23878C58646224E
:105C0700E54824F640EFE5580460EA75A700758378
:105C170007E559C42408F582E070DB0582E0FFE55B
:105C27004A64046015E54A6406600F801DEF24BED0
:105C37005029C23878C58646802175390AEF20E792
:105C47000975390520E6037539022038E0EF24C3CA
:105C57004009D23878C5A6467546001206E2A9BDA6
:105C6700E5597002A9BCE9240DC39F401F125B567A
:105C7700303D19753901204006D24078A876232097
:105C87005216E55965586010D233800C3033090538
:105C970059C233C240127ED622E558B4FF0122858D
:105CA700581175A704758307E54824F65002805CF0
:105CB700201259202905202A02805112B2AEE4F59C
:105CC70016F517751000125D2CE510700312B2A8B7
:105CD700125D45302910E51B2517F517F51BE51C47
:105CE7003516F516F51C125D5212B2A80510C3E55C
:105CF70011951050D175A70002B2B4E55AF51124D9
:105D0700F6500375110A75A70475830675100012FE
:0D5D17005D2C125D45125D520510C3E511B3
:105D2400951050EE75A70022E510C4F582E0E0F569
:105D340064E0F565E0F566E0F567E0F568E0F569CF
:105D44002275A70112606F12329D75A70422E9F033
:105D5400E51CF0E51BF022E510C4F582E0F512E540
:105D6400822406F582E0F511E0F51CE0F51B222003
:105D74002845E558B4FF012275A704758307E55942
:105D8400F510303306655860020510125D5BE0F5CE
:105D940013E07F797E3D12BC53E5137E3912BC5368
:105DA400E5127E3512BC5330480B7F7F7E3512C618
:105DB400AA0EBE40F9802C2012012275A704758317
:105DC40006855B10125D5BE512700B7E3A7F797479
:105DD4005D12BC85800D75F06484E5F07E397F7AB0
:105DE40012BBD5E53764027008304143127D5A80F6
:105DF4003EE51C7006E51B24FB5034E51164B460D9
:105E04002EA911E537600D200C0AC3E99570F950ED
:105E14000324B4F9E912C506781D79547D1D90C197
:105E24009FE53F20E00390C1A612C5F812BCB375EC
:105E34001779751619125E7075A7009006E3E511BF
:105E4400F0A31206E2E5BC75F019A4951BFBE5F07E
:105E5400951CFC922450031258A5ECF0A3EBF0C25D
:105E64004FEC7007EB24E64002D24F22E51C24EDF0
:105E7400402BAE1CAF1B1260397C007D3212572BB5
:105E8400C005EFAF17AE1612BB8ECE2405CE742C10
:105E940012BC850E0ED0E02312BB88801B1260302A
:105EA400125ECACE2405CE742C12BC85CE2402CE3A
:105EB400E875F0058412BC6BCE2404CE7422305DE8
:105EC40002746602BC85EE243D50047EC37F4B7C85
:105ED400017DF412572BC004C005EF6007AF17AE65
:105EE4001612BB8ED007D0067C007D3212572BA829
:105EF40005EFAF17AE16CE240ACE02BC6B1260308B
:105F0400EE2450305D03EE24A150047EC37F4B7C0D
:105F1400017DF412572BC004C005EF6007AF177E54
:105F24002F12BBDBD007D0067C007D3212572BC06A
:105F340005EFAF177E3712BC407E3B742C12BC5366
:105F44007E3DD0E075F0058402BC4020480122E487
:105F5400F5A7FC9006E3E0F9A3E0FE24FE40EFA3DE
:0E5F6400E0FF7D78E5376012304FE3200C1F20
:105F7200C3E99570F9501824B4F98013204F107DAD
:105F82003CE546600A7D141460057D0A1470C189DF
:105F9200111255FE7D6F12571EBE00B4EF24E2406F
:105FA200AFAD07E51112C506202404B2D5B2D178EF
:105FB2001F795612C5F8A806A907E511242D75F018
:105FC200B484E5F012C5067407304F02740EFDFA70
:105FD20012C5F8B2D5B2D112C5F8B2D5B2D1DDF040
:105FE200AD0212C5F8850616850717B2D5B2D112D1
:105FF200C5F885061E85071F7A03304F027A06E52B
:1060020011241675F0B484E5F012C506A816A91776
:10601200AD0212C5F8DDFBE51124EA400224B412F8
:10602200C506A81EA91FAD0212C5F8DDFB22E51B9D
:106032002402FFE4351CFE305D1ABEC305BF4D02CB
:106042008012AC06AB077A1B12562078321257C266
:10605200AE04AF032278737964125975125A8975A6
:106062001CC3751B4B2032048B1C8A1B22126057E7
:1060720030320122AC19AE1AA91DAF1FB90005BCFE
:1060820000028010C3E913F9EF13FFC3EC13FCEE17
:1060920013FE80E8BF29005006BE2900500122C32A
:0160A200EF0E
:1060A30013FFC3EE13FE80EB3E7FE3E3E3E3E3E39F
:1060B300E3E3E3E37F3E0C1C3C7C7C1C1C1C1C1CAC
:1060C3001C1C7F7F3E7FE3E3E3070E1C3870E0E395
:1060D300FFFF3E7FE3E3030F0E0F03E3E3E37F3EA4
:1060E300070F1F3F77E7E7FFFF0707070707FFFFD5
:1060F300E0E0E0FEFF030303E3E37F3E1E3F73E0C4
:10610300E0E0FEFFE3E3E3E37F3EFFFFE3E30303BC
:10611300070E1C38383838383E7FE3E3E37F3E7F91
:10612300E3E3E3E37F3E3E7FE3E3E3E37F3F030316
:1061330003E77E3C000000181818FFFF181818002A
:106143000000000000000000FFFF0000000000004E
:106153003FF00000381C38F00180C1F020F0FC0053
:1061630038F03FE0000000007CC6C6C6C6C6C6C6FF
:10617300C67C1838781818181818187E7CC6C60CF0
:10618300183060C0C6FE7CC6C6061C0606C6C67CA2
:106193000C1C3C6CCCFE0C0C0C0CFEC0C0C0FC06F2
:1061A30006C6C67C3C66C0C0C0FCC6C6C67CFEC66E
:1061B300C6060C18303030307CC6C6C67CC6C6C690
:1061C300C67C7CC6C6C67E060606CC7800001818B8
:1061D3007E7E18180000000000007E7E0000000094
:1061E30000000000000000000000000000000000AC
:1061F300000000008080A0C0A000304020C080804C
:10620300C0A0A0000060A0600000A040A05098D0F3
:1062130090882050A850888850A850206080600043
:10622300000040E0400000000000800000E00000AB
:106233000000000040002040800040A0A0A040409B
:10624300C04040E0C02020C0E0E0204020E02060CB
:10625300A0E020E0C02020C06080E0A0E0E020407B
:106263004040E0A0E0A0E0E0A0E020C0004000400B
:106273000000800080002060E0602000E000E0007B
:1062830080C0E0C080E0E0E0E0E00000000000400B
:10629300A0E0A0A0C0A0C0A0C040A080A040C0A01B
:1062A300A0A0C0E080C080E0E080C080806080A0CB
:1062B300A060A0A0E0A0A0E0404040E0202020A0FB
:1062C30040A0A0C0A0A080808080E0A0E0A0A0A00B
:1062D300A0E0E0E0A040A0A0A040C0A0C08080401B
:1062E300A0A0C060C0A0C0A0A060804020C0E040CB
:1062F300404040A0A0A0A060A0A0A0A040A0A0A05B
:10630300E0A0A0A040A0A0A0A0404040E02040808A
:10631300E02020A870202070A8202008F030D010A2
:106323000000F0A8A8000000E000000090204870E2
:106333008898984000E0E0E000A0E0E0E0406030B2
:10634300103060609090909090602060202020201A
:1063530070609010204080F06090102010906010CA
:10636300305090F01010F080E0101090606090803A
:10637300E0909060F010202040404060909060904A
:10638300906060909070109060000000000000002A
:1063930000000000000000506050007070500000CA
:1063A30078807008F000F8888888F800C0C810204A
:1063B30040981800C0B098B0C000602040000000B2
:1063C300000090D8FCD8900000246CFC6C240000E2
:1063D30020A870A82000002020F820200000000042
:1063E30000000080000000F000000000000000003A
:1063F300606000081020408000708898A8C88870EA
:1064030020602020202070708808102040F8F810A9
:0D641300201008887010305090F81010F81C
:1064200080F008088870304080F0888870F8081084
:10643000204040407088887088887070888878080C
:10644000106000606000606000000080000080005C
:10645000002040F84020000000F800F80000002074
:1064600010F81020007088081020002000000000A4
:1064700000000070888888F88888F08888F088880C
:10648000F070888080808870E09088888890E0F83C
:106490008080F08080F8F88080F080808070888034
:1064A000B8888878888888F8888888702020202094
:1064B0002070381010101090608890A0C0A09088B4
:1064C000808080808080F888D8A8A888888888887C
:1064D000C8A898888870888888888870F08888F02C
:1064E00080808070888888A89068F08888F0A09064
:1064F0008870888070088870F820202020202088EC
:1065000088888888887088888888885020888888C3
:10651000A8A8A8508888502050888888888850204B
:106520002020F80810204080F800CCAC9CACCC00B7
:1065300000CCD4E4D4CC0004781828C800FC40A0D7
:106540004018202018000000000000F800000000A3
:10655000A040A0000000600060600060006000607B
:10656000600000F0A8A8A8A820502000000000505B
:1065700090B890D090886050500070705080504813
:10658000FC485080304C5C6060603C00E0F00808E3
:1065900008F88044485C48448000882020887000C7
:1065A0000080C0A090F8003048B4B44830003048B3
:1065B000B4B44830FC0098D02058C8008080F088DF
:0A65C000888888F8E8D880D8E8F849
:0300000002005E9D
:03000B0002A12728
:0C000E00206E06859950D26E32D26F32FF
:0E00230010990AC298206DE385994FD26D3274
:10003800E4F537F534F520F52FC229C22AC268C283
:0800480027C214C2150221B900
:03005B00021FD8A9
:10A11A008530F0C5F065308530F060F722C0D0C0D8
:10A12A00E0C0F0C0A775A700C083C08275D00875CB
:10A13A008A3D758CEA0532E532700215320530E542
:10A14A0030640A6026201520E531B40C0BE530B4E2
:10A15A00010612A4AC12BFA6E531B4180BE530B45F
:10A16A00060612A4AC12BFA602A320C2AFD2C075C3
:10A17A00C07AD2AFF5300531E53164197045F53151
:10A18A00201522C22C7D0A740412C751EE24F54010
:10A19A00142402400E24014008202005DDE9021F94
:10A1AA00CCD225D22CE5A6600215A678A9E66001D4
:10A1BA001678B5E660011678B6E660011678D8E634
:10A1CA00600116302E09E5367005C22E12A433E559
:10A1DA00367004C24B8002153678A8E6600116056F
:10A1EA0035E53570021535E590307B0B30E008D245
:10A1FA0078C27BC200801A307C0B30E108D279C267
:10A20A007CC201800C307D0930E206D27AC27DC25E
:10A21A0002E59044F8F4700B753500302D05C22D17
:10A22A0012A433E5336005153302A2C5E590F45450
:10A23A0007700302A2C5F52075330820001B201001
:10A24A000C2011098013E59030E10E8006E53724D1
:03A25A00FD40F3D1
:10A25D00E543541FF53320100375A6FF78A8E6706B
:10A26D0057202D54202E51301004E536704A201001
:10A27D000C201109E53524F55003753304D21BD29A
:10A28D00A5D2A675B40C75B22278A77655C21C0559
:10A29D003420272420682120291E202A1BA2107279
:10A2AD00115015E5206011E5342438400B200026AF
:10A2BD00200119D27D7534C8201558E5317024124E
:10A2CD00C73174E812C70A802A02A3D9E53724FDE5
:10A2DD0040E6D27C80DF3011DFE53724FD40D9D256
:10A2ED007B80D275F00384E5F070DE12AFAE74E8BA
:10A2FD0012C70AE531B4060512B1318016B40C054A
:10A30D0012B147800EB4120512B1318006B4180394
:10A31D0012B147E59020E20620101020110D78A80B
:10A32D00E6704920103120113280562027F0206828
:10A33D00ED2029EA202AE7E534243140E1240450B8
:10A34D00DD90A36093D2A6201002C2A6D2A512A4BE
:10A35D0026804AC8A08267E5367011E59020E2217B
:10A36D00E54375F009A495355017D22DD2A62010CE
:10A37D0002C2A6D2A57418304B02746412A42680B2
:10A38D001C20340E305A08E54A603C141460381213
:10A39D00A433101B08A25892A5A25992A675A70026
:10A3AD00D082D083D0A7D0F0D0E0D0D0202006C569
:01A3BD00A6F9
:10A3BE006003C5A632201003021FCC7581D87438F5
:10A3CE00C0E0E4C0E03212A3F180C6C218B40202AB
:10A3DE00D21812B04C30180874E412C70A02A30047
:10A3EE0002A2FB78A7E66002162230754079AA77A2
:10A3FE0000E579602C14FF760D24CE4006EF90A474
:10A40E007A93F6301C1FEF249C7410400BEF240A35
:10A41E0075F0DFA4746F95F0C21CF5B4C313F5B2DA
:10A42E002278A7767DD21CE4F5B4F5B222E5792424
:10A43E00CE50097628301CED741480DC79A1E579B4
:10A44E009740E2E57979AAC7272464200E03F42405
:10A45E002CFF301C06EFF6243680BDEF200D02C314
:10A46E0013F6EF300D022436D21C80AE78726D6872
:10A47E00635F5B57534F4B4845423F3C393734324D
:10A48E00302D2B2928262422211F1E1D1B1A191898
:10A49E001716151413121110100F0E0E0D0DD2B536
:10A4AE00C28EAE8DAA8DAF8BAB8BE4F58DF58BD2B4
:10A4BE008E3014012278B6BE0007EF24E2400280EF
:10A4CE000806E624EC50027614E624F64005E4FE77
:10A4DE00FAFFFB7C007D0A1255FE7C007D5E125752
:10A4EE001E8F7EEE6003757EFFEAFC7A33125612E3
:07A4FE00EBF5F0A4E5F0CB43
:10A505008CF0A425E0C5F035E0CB926C25F0500623
:10A515000BBB0002D26C30E7060BBB0002D26CEC21
:10A52500F5F0A42BFBE5F03400FC306C010C78A6AB
:10A53500E6C39BFF18E608F6EB18F618E69CFE182E
:10A54500E608F6EC18F6301401227A0050040A12D7
:10A5550058957C007D6E12571E8FF078A2E6A4FBFD
:10A56500ACF0125834EBBA0002F404FAE4F8FFEA4E
:10A5750030E70118E57960062075031FF4042AF514
:10A5850079EF38D27520E70860037579FF02B26A62
:10A59500C2750470F5E579F40460EFF57980EE1283
:10A5A50006E2E5BE78A2F624F65007E4F5BEF612FB
:10A5B50040891206DD85BC2B85BD21E5BEF5482405
:10A5C500F65008E4F5BEF548124089E5BFF5432489
:10A5D500F8503B24F340371206D878A1E5BCF624A1
:10A5E500CD50087432F5BCF6124089E5BD24F6500D
:10A5F5002824914024E5BF789DF61424FB50087467
:02A6050003F65A
:10A60700F5BF12408978B7A6BED25322740AF5BFA8
:0FA61700F54312408980BE75BD0F12408980D473
:10005E0078FFE4F6D8FDF478D8F6F5A6D220D2B41F
:10006E00D2C075C07A75D75075AE1375AF01758154
:10007E00D875A882D2BC758951D28C7590F875EF5F
:10008E00BC75FDFFC258D25912A5A4D2A412C681C6
:10009E00C2A412A62612C73112AF24C22012C05912
:1000AE00121EA27F527E01908A031265E2123F8ACF
:1000BE0012C5AF12C681745012A42612C68112A4A4
:1000CE0033123AB812C05912C40F12C5AF12C67A03
:1000DE00753A00123B0AE53A701612C7657F437EE9
:1000EE0006908F711265E212C5AF12C674021FCC54
:1000FE0075A6FF123AB812A5A4121EA212C5AF120F
:10010E00C67DE478B5F678A9F6F52012C05912AF7F
:10011E0019C215C214121EA2908A227F781265CAC5
:10012E00205E0A7F767E12908A2F12BCB37F401219
:10013E00C58B7F497E0E78AEE612BB887E18743B67
:10014E0012BC857E1BE53E12BB887E25743B12BC1D
:10015E00857E28E53F20E00805A6E5A6700215A6D7
:10016E00E53F12BB887F5312B4687F577E0B12BADD
:10017E004A12BAD27F603073647E0BAC5DAB5C12F8
:10018E00BA4E12BAD27E3112666D7F6A7E1212BEDE
:10019E00F47F727E05743A12BC53E5A675F01E8488
:1001AE00A8F07E0112BC40E53F13E8337E0812BB77
:0701BE00D512C5AF10003699
:1001C500100136100236123A56D2AC75369612C464
:1001D500BEB4E005123B50800AE53670F1123AA62E
:1001E50012C67A0201192074097E2BE52E540712D6
:1001F500BC727E17809A021FCC02218C8078E5356F
:1002050024C8504FE59020E24AD0E0D0E0120259D0
:100215000251DDE53524D2503AE59020E235D0E0B3
:10022500D0E012C765803EE53524D25026E5902002
:10023500E221D0E0D0E012C765306B11908C577F7A
:10024500091265CA12C5AF12424D126A5C120259F3
:1002550002037A2212C765908FF77F001265CA12D2
:10026500C5AF02C67A12C765908FF77F001265CABF
:1002750012C5AF12C67DC215C214C227C268E4F505
:1002850035F520753701908AB712120690029573DD
:10029500020101020D050204590213E302037A0269
:1002A50003B90251DD0203050202B01002C81001B4
:1002B500051000C280F510020D1001BA1000028071
:1002C500F512409480B0D25312C765F54BF54C1228
:1002D5003A46E54B12C313054BE54C12C313154CB7
:1002E500D2AC7F3C12C4BE7E0512BB3A12C4BE7EA0
:1002F5002312BB3A12410112C6853000D202027B9D
:10030500E4F535F520753707908DC8121206900370
:10031500177302027B0203F602042302033502036C
:1003250005020305023DB0023FBB02033A02034545
:10033500123B0D801C123F4B12407A12C05980C0EF
:100345007F52A25E120598925E1205B380B21240EA
:1003550089E4F535F520753702908EF21212069074
:1003650003687302030502070D0207720207C9023B
:10037500080D020851C268E4F535F520753705907A
:100385008BD312120690038E7302027B0268200241
:1003950068650269FA02037A0203B20269390269E1
:1003A5009F020CCE02037A020CB40205227F2E12A4
:1003B5000C1C80C1E4F535F520753706908C90123C
:1003C50012069003CB7302027B020D0B020D650230
:1003D5000DD8020EA5020ED7020F4E0203B9020375
:1003E500EC020F810210267F49120C1C80C61240B8
:1003F50089E4F535F520753703908E1A12120690AB
:10040500040873020305020A6302054302054E024E
:100415000AC5020C62020ADD0205BF124089E4F535
:1004250035F520753704908E9B12120690043573AE
:1004350002030502055D02056802057302057E02D9
:1004450005890208600208A902093C020996020909
:10045500CF020A19D25712C7651212E412046702B5
:10046500027B7F177E02908B091265E27F4C7E022C
:10047500908B201265E2AC5DAB5C7F577E0412BAAF
:10048500CA1206F185BC6285BD637F377E0F74464F
:1004950012BC857E15744C12BC85E560240FFBE407
:1004A5003561FCA25C923BD25C7F377E1E12BA4E50
:0B04B500A23B925C7E30742012BC85DC
:1004C0007E36742012BC85E5602562FBE5613563EC
:1004D000FC7F227E0412BACAE56245637015742E51
:1004E0007E3A12BC8512C5AF10000C100114100228
:1004F00025809C742080E91562E562B4FF0C1563C9
:1005000080080562E56270020563E53524F5500355
:1005100075330102048F1206F18562BC8563BD024A
:10052000408912134D12C5AF10001510010280F85A
:100530007F637E05908C571265E212C5AF12421C94
:1005400002037A7F13A20D120598920D80097F1C79
:10055000A20E120598920E1205B30203F67F0AA2AC
:100560000F120598920F802A7F13A2081205989205
:1005700008801F7F1CA20C120598920C80147F2506
:10058000A20B120598920B80097F2DA209120598E3
:1005900092091205B30204238F1F92171207051246
:1005A00006DD85BC2B85BD21AF1F1F7E391272B0C1
:1005B000A217221206DD852BBC8521BD02408920B1
:1005C00037141206D885BE121205EC1206D8851211
:1005D000BE12408980057F3F1205DE0203F67E03CE
:1005E000908E631265E212C5AF02C67A75A6FF123D
:1005F000C76512A11A740712C7518FF0740612C78B
:1006000051EF2512C395F0FD78D8E6C4540F2DA202
:0E061000E7923D4010FD24CD50027D32AC0536
:10061E00C3743F9DFD800FF404FD24C850027D3746
:10062E00AC0574402DFD7F4012B4607E1212C6AA36
:10063E000EBE1EF91F303D020F0FEF6D70EDE53649
:10064E00700A753606EC2513F5148C131206731208
:10065E00C5AF1000071001083002072215128002E4
:10066E0005120205EC7F377E28742E12BC857F346E
:10067E007E21740A303D010412BCA2E514FC249CB8
:10068E0050027C63EC75F00A84C0F07F347E2D122C
:10069E00BCA2D0E07F377E3612BC727F437E1E1224
:1006AE00BA4A7E00E51212BBE17F057E02908E6F84
:1006BE001265E27F6D7E01908E7A1266157F747ED2
:1006CE0004908E8C1266150212E475C6F8802175A0
:1006DE00C6F9801C75C6FA801775C6FB801275C6E2
:1006EE00FC800D75C6FE800875C6FF800375C6FDBD
:1006FE0075C70375B90122743F12BC5302C5AF7F93
:10070E000A1207057E2A123B0D1206E2A8BF120737
:10071E004110001210010510021580F508E824E7BB
:10072E0050EC781880E818E830E7E3780080DF882E
:10073E00BF80627F097E059090AFB80C03909058F1
:10074E001265E27E27E53D28240C75F01884E5F04D
:05075E0012BB1D7E33FB
:10076300743B12BC857E35E53E12BB1D02C5AF7FCF
:10077300131207051206DD85BC2B1207A61000080D
:1007830010010510021780F2105C07205D0BD25C8C
:1007930080E8105DE5D25D80E1D25C80DD852BBC15
:1007A300020353205C10205D189090B57F127E23C6
:1007B3001265E202C5AF9090C9205DF09090BC80B5
:1007C300EB9090C280E67F1C1207051206DDA8BFDE
:1007D30012080010000810011110021A80F2E82418
:1007E300F750031880EA780880E6E824EC40030811
:1007F30080DE781480DAE8F5BFF54380A37F1B7EA3
:100803002EE8232312BB2302C5AF7F25120705124F
:1008130006ECA8BCE812084812C5AF100008100186
:100823000D10021F80EEE824E050E9188006E8244A
:10083300CF40E1081206EC88BC124089D21512C0E1
:100843005980D180157F247E3724E202BB8E7F2E10
:10085300A20A120598920A1205B30203567F3712B1
:1008630007051206D8A8BDE812089112C5AF1000FB
:100873000810010D10021280EE18B809EA7878808A
:10088300E608B879E2780A80DE88BD0204207F3664
:100893007E2975F00284C0F012BB23D0E075F00509
:1008A300A47E3B02BC727F3F7E1D743E12BC851248
:0A08B30006F1A8BF53001F53BFE079
:1008BD0012091F10000810010D10021480F218B853
:1008CD00FFEE781780EA08E824E850E4780080E02D
:1008DD007E1D745412BC8512091F7E2F743E12BCEE
:1008ED008512C5AF10000810011110021B80E8150C
:1008FD00BEE5BEB4FFE175BE0B80DC05BEE5BE24D2
:10090D00F450D475BE0080CFE8541F25BFF5BF024B
:10091D0004207F3F7E24E812BB1D7E30743A12BC4A
:10092D00857E35E5BE75F005A412BB1D02C5AF7FF2
:10093D004912070512096D53BF1F120978100008DF
:10094D0010010B10020E80F21853000380EC0853B7
:10095D00000380E6E8C42354E025BFF5BF02042060
:10096D001206F1E5BF54E0C403F8227F487E29E862
:10097D00600F9092041265E27E38E812BC7202C5D7
:10098D00AF9092081265E280F57F521207051206AC
:10099D00DD85BC2B1209BC100008100105100209E1
:1009AD0080F2105FEFD25F80EB852BBC0204207FBD
:1009BD00517E239091F0305F039091F71265E20222
:1009CD00C5AF7F5B1207051206E2A8BC1209F21033
:1009DD00000810010810020880F21880EF0880EC62
:1009ED0088BC020420E812B80B7F5A7E1AC31392FA
:1009FD003D12BB3A7E2C742C12BC85E4303D027442
:060A0D00327E2F12BB1D1A
:100A130012351002C5AF7F641207051206E2A8BDA6
:100A2300120A4610000810010D10021280F218B8C5
:100A3300FFEE787D80EA08B87EE6780080E288BD24
:100A43000204207F63E82312B80B75F06484C0F0BE
:100A53007E2612BC727E2C742C12BC85D0E080AB37
:100A63007F0A1207051206D8A8BCE8120A9712C516
:100A7300AF10001010010510021280EE18B8FFEA43
:100A8300783280E608B833E2780080DEE8F5BC7996
:100A9300A1F78072305C01237F097E2375F00A84FD
:100AA300C0F012BB8E7E2D742C12BC85D0E07E2F3D
:100AB30012BC6B0F7E359090CF305C0390912B026C
:100AC30066157F251207051206E2E5BE7F247E2CFC
:100AD300127305F5BE79A2F7802C7F371207051232
:100AE30006DDE5BC20E201E4540375F003A47F3680
:100AF3007E321273050475F0038460022404F8E562
:100B0300BC54F848F5BC0203F31206DDE5BE7F09C9
:100B13007E3A02BC721206E2A8BF1207411206DD3A
:100B230085BC2B85BD211207A6A8BF12080012069B
:100B3300ECE5BC1208487F2DA20A020BD51206DD94
:100B430085BC2B85BD217F12A20D120BD57F1BA265
:100B53000E120BD51206D8E5BC120A97A8BF120CC9
:080B6300A0E52B540375F0031B
:100B6B00A47F367E3212BC721206E2E5BE7F247E73
:100B7B002C02BC721206E2A8BC1209F2A8BD120A22
:100B8B00461206D8E5BD1208911206F1A8BF530014
:100B9B001F12091FE5BF54E0C403F81209781206AF
:100BAB00DD85BC2B85BD211209BC7F09A20F120B61
:100BBB00D57F12A208120BD57F1BA20C120BD57F6F
:100BCB0024A20B120BD57F2DA209744E400274592F
:100BDB007E3A02BC851206DD85BC2B7F51A25E805E
:100BEB00E9126C507F731268E6126C9F7F6C12686F
:100BFB00F57F2D800E1206DDE5BE7F097E3A12BC15
:100C0B00727F487E1E908C6B305303908C70026504
:100C1B00E21207051F120C0E12C5AF1000081001CF
:100C2B000510020980EF1053ECD25380E8221254C6
:100C3B008BEBF516F5147F6C1268F512546F7F640D
:100C4B007E23E51612BBF1C3E5169514F5167F73DB
:100C5B001268E67F2480AC7F2E1207051206D8A8F7
:100C6B00BFE824FA40033037027803120CA012C5F8
:100C7B00AF10000810010D10021280E518B800E14A
:100C8B00780580DD08B806D9780180D5799DE8F71D
:100C9B00F5BF0203F37F2D7E2C7420B80502742E52
:100CAB0012BC857E32E802BC72D26875480A123BD0
:0E0CBB000DD214122004126D8A1228E5C26BAD
:100CC90012022C80F3D214751501126C0A75B90140
:100CD900E5BC20E71C126D3A75A6FF126D9612133A
:100CE9000A12C5AF1266EA10000F50051268128089
:100CF900E70515E515242050D102037A120D1102DA
:100D0900027B120D110203B9120D1D1206DD854871
:100D1900BE024089121FF6122010125CA012C7658C
:100D2900908CF31275EC1275A41212BA12C5AF1099
:100D3900001410010510021B80F50548E548640AF6
:100D49007002F54880D11548E54864FF700375487D
:100D59000980C4854849122010E55822121FF685DA
:100D69004849C250E558B40F02D250125CA08038ED
:100D7900D22775480A122004125CA012C7651275A1
:100D890002908FB9202903908FC412136EC26A1280
:100D990028E5106A0280E1C227126BE285494812F0
:100DA9001135122010125CA012C765C2481275E9EC
:100DB90020500E12135812C5AF1000101001B18047
:100DC900F812130A12C5AF10000280FB0203B91210
:100DD9001FF6E55830E7137F1B908FA37E05126538
:100DE900E212C5AF12C67D0203B9122010125CA02F
:100DF90085594912C7651212F4908FC41275EC1205
:100E090075AE12C5AF10000810010A10020C80F56A
:100E1900120E7080DB120E7D80D612C7651212F495
:100E2900908D031275EC1275AE1275B212C5AF1022
:100E3900000810010A10020C80F5120E8980DB12DD
:100E49000E9780D61210FB122010125CA012C765F3
:060E5900908F371275ECCA
:100E5F0012133212C5AF10000510028880F802037A
:100E6F00B90559C3E55895595003755900221559BD
:100E7F00E55964FF7003855859220549D3E5491494
:100E8F0095584003754900221549E54964FF7005DF
:100E9F00855849054922121FF6E55830E7057F248A
:100EAF00020DE2122010125CA012C765908D0E1277
:100EBF0075EC12136312C5AF10000A10010280F80F
:100ECF001211A480DE0203B9121FF6E55830E705B0
:100EDF007F2D020DE2C26B7559FF125CA012C76520
:100EEF001212E4E55930E7031212FF908D1F1275AD
:100EFF00EC1275BE12C5AFE55820E70610000810BA
:100F0F00011110021B80F00559C3955950CF755927
:100F1F00FF80CA1559E55964FE70C285585980BDC6
:100F2F00E55920E711D26B75A700758307C4F582C9
:100F3F00E0B2E7F080A7306B031211520203B9122F
:100F4F001FF6E55830E7057F36020DE2122010122A
:100F5F005CA012C765908D2A1275EC12134D12C545
:100F6F00AF10000B10010280F81211991211CE026E
:100F7F0003B9121FF6E55820E7087F51908D340210
:100F8F000DE512C765908FCF1275EC12130A12C5BB
:100F9F00AF123A46D2AC10001FE55830E7F8306D6B
:100FAF00F51210AA7E207F005013908FE81266155D
:100FBF0012C5AF12C67D80CAC2AC0203B91B8B1318
:030FCF00908C57AC
:100FD20012661512C5AFC26B7B007514B812118E62
:100FE200126D09126CBB5025A814E824384004A6DF
:100FF2000105140BC3E5139B50E678B81211D030EB
:101002006B03126A5C122010125CA08082126C5078
:10101200E51660E6D26B126D66C003126C21D00336
:10102200A91580C4121FF6E55830E7057F5A020D54
:10103200E2122010125CA012C765908D3F1275EC6F
:1010420012132712C5AF10002410010280F81210EB
:1010520072908FDA5003908FE81275EC7F007E3C1D
:10106200E54B12BC4012C5AF12C67D80C40203B963
:10107200123A4612C345745212C378745412C313FF
:10108200E5580475590012C33412669A4016126B61
:10109200E2126D3A1266EA400B0559C3E5589559BA
:1010A20050ECC322C2ACD322123A46D2AC12C4B91B
:1010B200C5F060F0C5F0B440F412C4BEB4400312EF
:1010C200C4BEB452DFF53812C4BEB454D712C4BE83
:1010D200FA60D124EF40CD12C4BEE53870C612C406
:1010E200BE12C4BE12667F7B0012677240B6126DDA
:1010F200190B12667FDAF2C3221211DFE55924C8F6
:10110200F88602E54924C8F9986013146010500F5C
:1011120018E608F618E86970F7A7021211CE22E560
:011122005973
:10112300640F60F91908E618F608E86970F7A70272
:1011330080E81211DF78C8C250E6B4FF02800708C6
:10114300B8D8F6D25022B8D702D250A615807C78F0
:10115300B81211E1E4F9F5A7758307E9C4F582E054
:1011630030E70AE924B8F82438400276FF09C3E5DA
:10117300589950E712119978B879C8E6B4FF0280FC
:1011830002F70908E8243850F2804079B877FF095C
:10119300E9243850F82279C877FF09E9242850F860
:1011A300221211DFC23D78D7B6FF04A900D23D1841
:1011B300B8C7F5203D0279D81978C8B6FF0122C314
:1011C300E8995007C6C7C6081980F478C81211F009
:1011D300126D78126D78126D78026D7878C81211DD
:1011E300F0126D54126D54126D54026D5475C70391
:1011F300E54875F004A42480F5C62212C76512657C
:10120300CE800612C7651265D2E53760461460408A
:1012130014603814603014602814602014601814AB
:10122300600B14600814600A1460028026120BE03D
:051233008021120C39BE
:10123800801C120C008017120BEC8012120B7F809E
:101248000D120B408008120B188003120B0C12C5EC
:10125800AF12C6811212E4D234E4F5B4F5B2A81F75
:1012680008E814C23BB51D02D23B75F007203C03C9
:1012780075F009A4FF203C010F7E007420303B026A
:10128800743E12BC53D8DA12C5AFE51D1000081021
:10129800011010021880C0651F7003751DFF051D21
:1012A80080B57005851F1D80AE151D80AA75F003D9
:1012B800A4227F7B7E00909183126615E54824F670
:1012C80040087E0A908F85126615221269127E05E3
:1012D800745B12BC4F7E1D745C02BC4F1212D37E2D
:1012E8003490919402661512691280031212D37E0B
:1012F800319091980266151212D37E31908FF802C0
:1013080066151269127E0080051269127E2D908F73
:10131800F80266151213277E31908C750266151235
:10132800130A7E1A908C7A02661512130A80C0126C
:10133800130A7E18908C4402661512130A7E1A90BE
:101348008FFD02661512130A7E1A90900202661526
:1013580012130A7E1A908CFD02661512130A7E1863
:10136800908D190266157F007E2012661502C5AFA2
:1013780012691290900802661312A8BD1206FBE5C6
:10138800BDF55EF56CE5BCF55FF56B756A007561DA
:10139800FF75A70490070012A869B4FC12E582C380
:1013A80013F561E56CF0E56BF0E58260168005B435
:1013B800FF02800F12A7AFE56C655E70DAE56B651A
:1013C8005F70D475A70022E560758307C333F58283
:1013D800E0A3F56CE0F56B756A0022D214C21F1207
:1013E8001381756000E561B4FF1612C765908B2BF9
:1013F8007F0A7E0512661512C5AF12C67A02027BF5
:10140800C210C21112C7651212E4301F0A7F07907A
:101418008B3912661380647F007E01C3E56012BBBE
:10142800F17E0E742812BC4F8560487407F51FFFC3
:101438007E00743E12BC53E5481213D112B28612D4
:1014480019570548C3E5619548FD401CE51F240769
:10145800F51F24C850E17F387E01ED0412BBF17EF0
:101468000E742912BC4F800DE51F2407FF7E0190E2
:101478008FF7126615201F0312199A12C5AF1000B4
:101488001910012C10020280F5120218301F3D02BB
:10149800026A101F02D21F021408E56160F4E560B9
:1014A80065617005201FF080E9201FE6056080E770
:1014B800E56160DEE56065617005201FD580092063
:1014C8001FD5E560700280CA156080CB12138112A7
:1014D80013CF12B286121A8E756A1012A850121BF8
:1014E80045908B401265CE12125C9014F67302146C
:0414F8000802272C93
:1014FC0002151F02150212134D12C5AF1000C910B0
:10150C00010280F81213CF12A869C2E2FF12A6F0F2
:10151C000213E3C2531213CF12B286753700908BAD
:10152C0059121206901534730214D40217210217A3
:10153C002602151F02155B02156002151F02159E6F
:10154C000215A20215A60215AD0215B10215B512AF
:10155C003A738003123A5E780A12167E740512C32F
:10156C00111216BD12C32D1216F812A85012A87C17
:10157C0012A76D12A99312180ED5150C75150A1217
:10158C00170B12192112C32D100204E57F70DB0218
:10159C0014D4780A8006780480027801123A738099
:1015AC000D780A8006780480027801123A5E1216D1
:1015BC007E740512C3061216BDE54812C2F2742AD7
:1015CC0012C31312C31312C31312C32D1216F81223
:1015DC00A85012A87C12A76D12A99312180ED5153B
:1015EC004885481512170BE51C12C2F2E51B12C2F6
:1015FC00F2E51B2548F51BE4351CF51CE4A277929B
:10160C00E7A27492E0A27392E112C2F2AD75AC74CF
:10161C00AB73E57DC412163FAD78AC77AB76E57D48
:10162C0012163F12193F12C32D100204E57F709F52
:10163C000214D4540F2375F00584F8C3EB33FBEC80
:0E164C0033FCED33FDC3EB33FBEC33FCED332D
:10165A00FD20E713EB28FBE43CFCE43D12C2F2EC6C
:10166A0012C2F2EB02C2F2C3EB98FBEC9400FCED5F
:10167A00940080E88848121311E4F54AF549756A1E
:10168A002075150112A85012A76DD5150E8548159B
:10169A00E5492401F549E4354AF54AE57F70E574E0
:1016AA004012C378747812C313746312C313741884
:1016BA0002C3061218FCE56012C2F21213CF12B26C
:1016CA0086E53A12C306E53B12C306E53C12C30699
:1016DA00E53D12C306E53E12C306E53F12C3067492
:1016EA000112C2F2E54A12C2F2E54902C2F212132B
:1016FA00CF756A20E4F51CF51BF514F51375150171
:10170A0022753800E51412C2F2E51312C2F205136B
:10171A00E5137002051422123A738003123A491231
:10172A00131112185712C685756A2075150175A608
:10173A00FF754A0112A7F612A76D12A99312180E85
:10174A00D5150975151E12183212C68F121921E500
:10175A007912C2F2E57EC333500274FF12C2F2E577
:10176A00711217F312C2F2E57012C2F2E57B24ACD1
:10177A00FFE55F340912C2F8EF12C2F2E51520E064
:10178A0033857D56E412C2F2E52EC412C2F812C3A2
:10179A003C12C68F10021A305594744012C3137447
:0417AA004512C3130E
:1017AE00744F12C313744612C31312C33C0214D4E3
:1017BE00E5561217CDC4FAE57D1217CD2A80C2FB6D
:1017CE00C41217DA2323CB1217DA2B22540FFC2460
:1017DE00F650027C009017E9EC9322000001010103
:1017EE000202030303FA2440400A24804003EA3332
:1017FE0022D2E72274FF2220E703C3132224C02241
:10180E00E53F701F7F7B7E0078AEE612BBDBEE24D9
:10181E0004FE743A12BC53EE2404FEE53E12BBD510
:10182E0012C5AF2278AEE612C306E53E12C306E538
:10183E003F12C306E412C2F2E412C2F2740A12C2DA
:10184E00F274C012C2F202C33C744012C313745439
:10185E0012C378744E12C313E412C2F21218FC743F
:10186E001812C306E53D12C306E56012C2F212134A
:10187E00CF12B28678ABE60812C306E60812C3068C
:10188E00E60812C306E612C306E53E12C306121E92
:10189E0089E51212C306E51112C306740112C2F2D3
:1018AE00909019121949756A1012A850057F057F7C
:1018BE00787F12C2EB787B12C2EB787D12C2EB7886
:1018CE007712C2EBE4FEFF780712C2EB12C2EBE511
:0F18DE007412C2F2E57512C2F2E412C2F2E5739F
:1018ED00C333500274FF12C2F212C2EB02C33C7535
:1018FD00C70375C6FF75B901C217751D0085BC1CE0
:10190D0085BD1B85BE1A85BF19125598EE12C2F200
:10191D00EF02C2F2E57512C2F2E57412C2F2E5737E
:10192D0012C2F2E57812C2F2E57712C2F2E5761232
:10193D00C2F2E55E12C2F2E57A02C2F275A700E4C8
:10194D0093700122A312C31380F5AF1F7E0478ADEF
:10195D00E612BBD57E0C742C12BC537E0E18E6120B
:10196D00BBD57E1A78AEE612BBD57E22743B12BC77
:10197D00537E24E53E12BBD57E2FE54012BBDB7EA8
:10198D0037743B12BC530E0EE54102BBD5753200C8
:10199D001213CF12B286857946787A796412B29F86
:1019AD0074641259738E47121A8E756A20D23D12C5
:1019BD00A85012A87C121AC5303D09307406C23DDC
:1019CD008E1E8F1FE57F602BE54C24FFF54CE54DFA
:1019DD0034FFF54D454C600512A78580D2751D3C31
:1019ED0012A85012A87C12A76D121AC5E57F6003CC
:1019FD00D51DED121B26901B3E12BCB3203D0DAE26
:101A0D001EAF1F121B26901B3712BCB3E546FD708F
:101A1D000B909153305D1190914F800C047010908C
:101A2D00914F305D0390914B7F3812350A804BE416
:0E1A3D00FFFC7E05305D047E027FB312571E53
:101A4B00AC06AB071255E87F38C23DE51C6007D2E8
:101A5B003D7E2C12BC40E51B203D026007D23D7E33
:101A6B003012BC40E51A203D026007D23D7E341295
:101A7B00BC40E5197E3812BC4012350FE53224C844
:101A8B0050FA22E54075F03CA42541FFF54CE435B6
:101A9B00F0FEF54D7C007D1012572B0F8F4BAF4C8A
:101AAB00AE4D7C007D3C1255FE7C00AD4B12572B8E
:101ABB00EE4F70010F8F4C8E4D2278647973C2D12B
:101ACB00121ADCFF78677976D2D1121ADCFE02C6C5
:101ADB00AAC3E796FB0809E796FC0809E796FDA25F
:101AEB00E7921750031258AD75135A30D10E751378
:101AFB0020B217AA47125632AB04AC05E546600B71
:101B0B0004600BAA46125649EB03FBEB03FBEB54A9
:101B1B003FFBE5132B2017029B9B22EE141430E79F
:101B2B0001E4FEEF141430E701E4FF220505708891
:101B3B00A8887005052020F8202075320012C76593
:101B4B007E1E7F1C12C6AADFFB12C6AA7E1E7F1C3E
:101B5B0012C6AADEFB7E1D7F1D12C6AADEFB7F000E
:051B6B007E2178ADE6CB
:101B700012BBD57E29742E12BC537E2D18E612BBE3
:101B8000D57E35742E12BC537E3918E612BBD57F34
:101B9000077E21745412BC537E25744F12BC537EB1
:101BA0002D78AEE612BBD57E35743A12BC537E3921
:101BB000E53E12BBD578AE121E897F0E7E21744C95
:101BC00012BC537E25744112BC537E2DE51212BB0C
:101BD000D57E35743A12BC537E39E51112BBD57FE0
:101BE000157E25744412BC537E2DE54012BBDB7E6E
:101BF00035743A12BC537E39E54112BBD57F1C7E49
:101C00002F85715412B8D67F217E0190911E1266E5
:101C1000157E0EAC77AB7612BA877E2B85795F8501
:101C2000787B12BF4D7F287E019091221266157538
:101C30001D2B751E10E574121E3D7E25742F12BCDF
:101C400053751D2D751E2BE575121E3D7F2F7E02CF
:101C5000909116126615E5736003121CEA7F367EBA
:101C60000290910E126615E572121CEA121D821284
:101C700013CF756A209004E6E56CF09004E7E56BFD
:101C8000F0AE4DAF4C7C007D4012572BBF00010FD2
:101C90000FAC07AD07E4FED23D12A85012A87C128B
:101CA0001D2BE57F602CE54C24FFF54CE54D34FF02
:101CB000F54D454C600512A78580DE751D3C0E1262
:0A1CC000A85012A87C121D30E57F29
:101CCA00600612A76DD51DED121D007F7812B47241
:101CDA007F767E00743012BC53E53224C850FA2253
:101CEA007E2112B80B12BBF17E2F909126305D0334
:101CFA0090912B0266159004E6E0FD9004E7E0FC63
:101D0A00C3E56A9420FBE56B9CFCE56C9DFD5003E2
:101D1A002410FD12581D9004E8EEF09004E9EFF04B
:101D2A0022DD03AD040E7F78E55E20E72AE57A8599
:101D3A0049F0A4A9F0E57A854AF0A429F9E435F036
:101D4A00FAE55E8549F0A429E435F02AFAE55E85CC
:101D5A004AF0A42ACF9FFF12C6AA103D18C3EF9BD0
:101D6A0050131BEF6B600E8F018B0712C6AA1FEF71
:101D7A006970F8AF01AB07229090D3305C03909062
:101D8A00EC754A40754900AF76E577FE20E76B703F
:101D9A0005EF24105064EF24A8EE34FD4011909012
:101DAA00D8305C039090F0754A1975499A8075EF9E
:101DBA002450EE34FB40119090DD305C039090F596
:101DCA00754A0C7549CD805CEF24A0EE34F64011BB
:101DDA009090E0305C039090FA754A0675496680E7
:041DEA0043EF24F0AF
:101DEE00EE34F140139090E3305C039090FF754A0F
:101DFE0004754944802A8028EF2490EE34E840117F
:101E0E009090E6305C03909104754A0275498F807C
:101E1E000F9090E9305C03909109754A0175499ACB
:101E2E007F401266137F4612B4727F5F02B472AEA9
:101E3E001E75F064305C0375F03284C0F0F87004E7
:101E4E00EE2404FEE51D12BC53EE2404FEE86007EA
:101E5E0012BC40EE2404FED0E075F00A305C03752F
:101E6E00F00584A8F012BC40EE2404FE742C12BCC3
:101E7E00530E0EE8305C012302BC40E53E2541F5D1
:101E8E001124C45003F511D3E63540F51224E85061
:101E9E0002F51222D23412A433C21012C7657F0586
:101EAE007E099089FA1265E27F137E08901EDE127B
:101EBE00BCB37F2B7E01901F4612BCB32037107F20
:101ECE00277E29E53F20E0010E901FB812BCB322F9
:101EDE00113007FE1FE001E101F80F00061B00F8AC
:101EEE000C00180E007C10007006003C2000E0066E
:101EFE00003E4001E004001E8003C004001F0003EA
:101F0E00C004000F00078000000F8007800000173C
:101F1E00800F00000027C00F00000043C00F00100C
:101F2E000083E00F00200301F00700C00F01F8034B
:101F3E0083007F87FE01FC000E3E180000030000A8
:101F4E000000180000030000000038000000000030
:101F5E0000003000000000000000FC761F0E1C6028
:101F6E0030ECFCBC3F172DF0F978613866264F61D6
:101F7E009A706070C60E1EE330E06060C60C1CC323
:101F8E0060C0E0618C0C18C7C0C0C0E18C1C39C6A3
:101F9E0011C0C4C19C9931963180C8C1FF1E31E772
:101FAE00E180F0C0EE1C31C3818006163091882886
:101FBE0092884924904927909248A0E3C8BCC2AFAA
:101FCE0074FE12A4267F6412C691C2B480FC75C73B
:101FDE0003E54875F004A42480F5C6C23C75B9012A
:101FEE00E5BC047002D23C221206DDE5BEF54824A3
:101FFE00F65003754800753400753703C228D22990
:10200E00D22A75C703E54824E75003754800E54812
:04201E0075F004A4B1
:102022002480F5C6751607751700C23C122051129E
:1020320020511220511220518517581558755900F8
:10204200E548B40A09E5586005F460020559222002
:102052003C1D75B90105C6AABCABBDACBEADBFEA9D
:10206200122072EB122072EC122072ED12207222F8
:10207200203C07F515B4FF03D23C22C0C7C0C612EC
:102082006C0A75A704851683E517C4F8F58275B93D
:102092000105C6E5BCF0C582F82406F92403C58211
:1020A200E5BDF0E5BEF0E5BFF075B90105C6E5BCDA
:1020B200F0E5BDF0E5BFF08516838982E4F075B9DD
:1020C2000105C685BC1385BD14E4F0F08882E5BE27
:1020D200F0E5BFF075B901E5BCF0E5BDF0E5BEF095
:1020E200E5BFF0758306E51723541E24B0F582E59B
:1020F20013F0E514F075A700D0C6D0C70517221259
:10210200A5A478BEA64808E4F6F55908761808F69C
:10211200C249C23608760A08F6060876BEC225C249
:1021220054C25512A8D2122004C229C22AC227C2FE
:0E21320068E4F537F52EF534F536F52F78A86C
:10214000F678AAF678B6F678B5F6789EF678B8A658
:102150005E08A67AC26BC233C238C240C223C22212
:10216000D24175460278C5A646C23AD221C219C2EA
:1021700026C23485705778BA7401F608F608F60856
:10218000F6E4F542F541F540220201011221011267
:1021900073D1754403123B0A129A1AD54403021FE5
:1021A000CC201EF1789F7680754A0012A663D2106B
:1021B000754E50C211C213C21212C059123A56C201
:1021C0004675A60A12AF1920120312267FE5A6242F
:1021D000FA4006123AA675A60A20251FE590540576
:1021E0007008E53524E250158011E54375F00AA426
:1021F000242295355007E59020E202806E201E1DB6
:10220000E532241040172046142428500D30410A8E
:10221000E537B40205127BA6D2461228E5D2AC30CF
:102220006DAB12C4C3B4E0A5123B50304108E53792
:10223000B40203127BA612234E1228E512920D124D
:10224000AAA01228E51273D130121D12AA8C12A76F
:102250000AE5510404F57F24FE4003757F02C2772E
:10226000E54024EF5002D2550221B975A6FFC210F5
:1022700030120BD221123B2E12A70A122286C21252
:10228000752F0002010112A8A912C765E47E057F1F
:042290001E908F7B92
:102294001265E212C5AF12C67DD214D2201206DD39
:1022A400852BBC8521BD75B90575B90212A8B3D2B9
:1022B4005512A7A97F0012A6F0D22012A8B3E56A8E
:1022C400600512A76D80F7857A62D2201206FB851D
:1022D400BEBC85BFBD856BBE856CBF75B90575B9C0
:1022E4000285BD6C85BC6B756A2012A8A91224F303
:1022F40012A7E812A8B3756A0012A850E57064FE2C
:1023040070437570FC854077854178851F7978180E
:10231400797A12B29F12A7527FB412A7D4D2201294
:10232400C68F12A8B3756A1012A8508554717F081D
:102334007810797212B2A185627C855E7D12A752F3
:102344007FC412A7D4C220C21422300A0122123A36
:102354007312249F745212C313744D12C313744323
:1023640012C3131224AE12C34E7441207402745665
:1023740012C3131223FB12244512C34EE53C12C3AD
:1023840006E53B12C306E53A12C30612247B12C3C8
:102394004E744512C3131224E412249F744712C3CB
:1023A40013744712C313744112C3131224AE1223BD
:1023B400FB12C34EE43074010412C31112C34E90D5
:1023C40004C3E012C30612C34E9004E4E075F00A9D
:1023D40084AFF012C30612C352EF12C311AC5EAB4A
:1023E4007A1224C0AC5DAB5C1224C012C34E12C37B
:1023F4004E1224E4023A567875C23D1224067878C7
:10240400D23D12C34E1270B6303D05E51E12C31103
:05241400E51D12C311DB
:10241900122488E51812C311E57D203D01C4540F2B
:1024290012C31112C34E303D097445301702745757
:102439008007744E301702745302C31320740812B4
:10244900247B12247B802775A7049004BFE0FCE05D
:10245900FB7A1B12562078321257C21255E8122401
:10246900859004C1E0FCE0FB1255E812248575A7AC
:10247900002212C34EE4F51AF519800D12C34EE578
:102489001C12C311E51B12C311E51A12C31112C3A1
:1024990052E51902C311742412C313744712C37885
:1024A900745002C31312C34EE53D12C306E53E1232
:1024B900C306E53F02C30612711212C34EE51D128F
:1024C900C313781CE612C31118B817F812C352E4E3
:1024D90012C31112C34E744D02C313C038742A12A9
:1024E900C313D03812C32D02C68F78107F0EE4F6BD
:1024F90008DFFCF564F565F567F5687515FC751A6F
:10250900C0751DC0756640756940754A0112A7F608
:102519003055030225AF12A76DE571B510004002D1
:10252900F510E57EB511004002F511E5122075029E
:10253900E513C395795006207545857913D3E57A56
:102549009514E5156480FFE55E64809F400C857AEB
:1025590014855E15857B16855F173074ADC2D178F9
:0D25690064797312258D7867797612258DBF
:10257600D2D17818797312258D781B797612258D2C
:10258600808B85791280B9D3E7960809E796080902
:10259600E66480FFE764809F20D101B3400AE7F636
:1025A6001819E7F61819E7F622E51AB4C00E78737B
:1025B600791812B29F7873796412B29F7818796489
:1025C600C2D112262074181259738E47AE1EAF1F41
:1025D600781B7967D2D1122620C3E51F9FE51E9E80
:1025E60050048E1E8F1F7EFF7FFFAC1EAD1F12573D
:1025F6002B7A04EF8AF0A4E5F0CE8AF0A42EFEE44E
:1026060035F0BEFF011E60051460057EFF8E1F2299
:10261600EE7E0020E7F77EFE80F3C3E697FB08090F
:10262600E697FC0809E697FD1818191930E7031212
:1026360058ADC3EB33FBEC33FCED33FDEB33EC333E
:10264600FBED33FC30D105AA471256490BBB0001FE
:102656000C751E03751FFFEC24FC40048C1E8B1F9B
:01266600E68D
:1026670027FB0809E637FC0809E637A2E713F6183F
:10267700EC13F618EB13F62210131978B5E624FAC3
:10268700401AE57124F64008E57924F640028034C3
:102697000606803012C68BE59030E2DFD220753611
:1026A70012D22EE4F534F537F55A12A9041226D1C1
:1026B700C219C257127ED6127F03853F4DD2122010
:1026C7005E02D228122173C22022D214122721E6D9
:1026D700F008DFFB857A621227177570FE783A7962
:1026E7007112B29F12A75212271785627A855E7BF5
:1026F7001206F185BC7E85BD7F7570C012A7521288
:102707002721E0F608DFFB75A700757F01C21422B9
:1027170074FF7870F608B880FB2275A7049004F060
:1027270078707F10221213CF12B28612AA2090045B
:10273700EAECF09004EBEBF0123A49751F0312181C
:102747005712C68BD51FF712210112C76512C5AFE5
:10275700C25AC258C259756A2012A7F61259718E09
:1027670047754A01753901C210D211D214D236D237
:102777001212A904127ED6127F0312C05975A6FF42
:10278700753609753200E59054057008E53524E281
:0A279700502E8011E54375F00BA4ED
:1027A100241995355020E59020E21BC211C2121266
:1027B100C76512C5AFE4F535F52FC22D7E0612C6E9
:1027C10087C2020214D4E54A20E01612AA03123A83
:1027D1004912C345744912C378780412C2EB12C37B
:1027E1002DC221E54AB40202D22112A7F612920D9E
:1027F100302612125D021273D4753606E53670FC6E
:10280100C2260227811273D11228E5E54A20E02170
:10281100B40209753900E53670F980E6E53960E200
:10282100FD24E24002053912A7F62026C6DDF88014
:10283100D1753900123A49D2ACE536602712C4BECF
:10284100B440F612C4BEB4400312C4BEB44915F577
:102851003812C4EEFC12C4EEFBAD3812C4EE6D703A
:1028610003122869C2AC809AC39004E9E0FF9B90EF
:1028710004E8E0FE9C50048E048F038C148B137AC1
:102881001012562074202BF56A9004E7E03CF56B9A
:102891009004E6E03D540FF56C754A0112A7F6AEBF
:1028A10014AF137C0E7D1012572B8F40AE04AF0571
:1028B1007C007D3C12572B8F418D429004EBE0252B
:1028C10013FF9004EAE03514FE7C0E7D1012572BA5
:1028D10078AEA607AE04AF057C007D3C12572B8F66
:0D28E1003E8D3F2210002910010D10020D48
:1028EE0020783020790A207A1722022A550229B53B
:1028FE00E5376006146006022ACF022A69022AA76B
:10290E000229D9E53724FD500A24FD4003022B3D50
:10291E00022B0B20115BE59030E25575340020122E
:10292E0003D2132278A9E6701FE5377005106B02EB
:10293E00D26B760AE53724FE40027603D277D22692
:10294E00753614D22E02A8F9200B25204122E53728
:10295E00B4021DE6B4050B127ED6127F0375360A3D
:10296E008009B4080B127ED675360578A916D22EBC
:10297E002210780122753900E53424384007754A53
:10298E000175340022700AE54A30E0F2754A028081
:10299E00F0146008754A06127F038006754A041209
:1029AE007ED675390180DA302909C229D22A7559A5
:1029BE00008005302A0CD22912759A12756875346A
:1029CE000022206847302703D26A22D222122CD648
:1029DE00107A0122C249E534243840077537007554
:1029EE003400227009E4C53770F5053780F1C24115
:1029FE00F5371470040537D241305E0B24FB500EB0
:102A0E00753706D22880D875370280F78033E537C0
:102A1E00640260CBC228E53724FD2324BEF879C4B6
:0B2A2E00E7F9A74809A75979C4E8F7A9
:102A39008648088607E537B40405754818D249124F
:102A490020108F59809E122CB2022C5CE537601041
:102A590014604B14607024FC4003022BB4022B8ACF
:102A6900D22312345810790122E5342438400775ED
:102A7900460175340022700EE54624FE40F1E54614
:102A890060ED154680ECB40600500C04F54624FAB6
:102A990050E075460580DB100FD8D20F80D4D223C1
:102AA90012345810790122E53424354012240240A9
:102AB90007105B27D25B8023100820D208801C10E6
:102AC9000C19D20C801510790122204127D24BE52F
:102AD900342437400AC25AC258C25975340022D226
:102AE9005A7006D258C25980F2C258D2591460EBB2
:102AF900D25880E778B8A65E08A67A753605D22E30
:102B090080D930122B1275D4055BE55B75F00B8407
:102B1900E5F0F55BE55A24F64009E55A955B500363
:102B2900755B001275D812C5AFE5346003D534D290
:102B390075340022C240302907022C22D23680F097
:102B49001049F91275961275AA102A29C233055926
:102B5900C3E55895595008755900E548B4181BE55F
:102B690058B4FF037559001275BE12C5AFE534603C
:0A2B790003D534C02275590080ED29
:102B8300D22A12759A80E93012231275D4155BE5A7
:102B93005B30E70C755B0AE55A24F64003855A5B04
:102BA3001275D812C5AFE5346003D534DA75340035
:102BB30022C2402029471049891275961275AA101E
:102BC3002A22C2331559E55930E71C855859E5586F
:102BD300B4FF03755900E548B41802800AD22A12DB
:102BE300759A800E855859E558B4FF03755900123C
:102BF30075BE12C5AFE5346003D534B5222010622B
:102C030020115F7F180548E54864187008F54830BF
:102C1300270375480A121FDC303C2DDFE88026208D
:102C2300105A2011577F181548E54830E7057548B5
:102C330017800A64097006302703754817121FDCD2
:102C4300303C05DFE275480A122010125CA0E53221
:102C5300244C500512756880031275027534000206
:102C6300C5AF122C997F0EE5486B70048A48800229
:102C73000548121FDC303CD0DFED80CC122C997F4D
:102C83000EE5486A70048B4880021548121FDC3039
:102C93003CB6DFED80B27A007B09E537B40301224D
:102CA3007A0A7B17B40501227418FAFBF5482275DA
:102CB300A704758307E559C4F582E0E0F573E0F5F1
:102CC30074E0F575E0F576E0F577E0F57875A70043
:082CD300025CA0E59020E27A0A
:102CDB00E534243750747F33122D60908A670F12BE
:102CEB0065CA7F3C122D60908A710F1265CA7F45B1
:102CFB00122D60305E30908A7A0F1265CA7F4E12A9
:102D0B002D60908A830F1265CA7F57122D60908AAF
:102D1B008C0F1265CA7F60122D60908A950F126519
:102D2B00CA7F69122D60E53424377F35601D147F0F
:102D3B003E6018305E15147F476010147F50600B97
:102D4B00147F596006147F626001227E2674711213
:102D5B00BC8502C5AF122D640F7E2F12C6DADEFBC7
:032D6B0002C6DAC3
:1073CE0002747E12C765E53724FD40F4E537B4023A
:1073DE000C304109E532248C50FA027BB012C37D89
:1073EE0012B81912B8B512BA4612BD427E197F36BE
:1073FE0012B94D12C25512B963E5376005146038E3
:10740E00805AC23A1275231234B11231DB30282061
:10741E001235881237DB1243A7E5486418600CE575
:10742E004824F65006201E031238C412C645801E8C
:10743E001237DB12358880DED23A12753BC23C120F
:10744E002D7412351C12B43F12B39D12C65D12C1BB
:10745E0003125ADB125D73125F4F800C12752F12DE
:10746E00B2EB12BEF012C635127B4812B935800748
:10747E0024FD401C12750275A70012C2CD302205E4
:10748E00122CD6C222302305123458C22302C5AFA5
:10749E001212E475170012C1AD7F1212B4603012D1
:1074AE004A75100075A704758306125D5BE51075AD
:1074BE00F009A42415FFF5177E00E512602F75F074
:1074CE006484E5F00F12BBD51F7E0EE51112B8775E
:1074DE00751623125EA10510C3E55A95104006E5F8
:1074EE001024F550BF3012031275D8808A745D12C5
:1074FE00BC8580D53029051212BA80101212E430E4
:10750E00490A7F7B7E00908C571266151275E92012
:10751E002A7A0275BE301215305E1230500F027884
:10752E0042301209305E06200B03027E0C205E17DD
:0B753E00E537B4021230120E12B459EF
:107549007F1712C58B75172012C1AD2212BE3720C5
:1075590012012230510612B79002B57A02B7ECE453
:10756900FEFFE54824F6400D908F851266157E16BC
:10757900E54802BC40B40E06908F8B026615908FC9
:10758900931266157E12E54824F702BBDB7D208045
:107599000C7D3F302A077D633029027D3C7F0080C6
:1075A900247D2080127D3E800E7D3CE54975F007E3
:1075B900A42406800A7D3FE55975F007A42409FF34
:1075C90064027001FF7E1CED02BC537D2080027DA8
:1075D9003FE55B75F009A42416FF7E09ED02BC5353
:1075E900908C3A7E207F001266151275687E007FA6
:1075F9000690769F12BCB3E5580460677510007554
:10760900A704758307125D5BE51075F007A42409CB
:10761900FFF5177E00E51212BC537805EE2404FE2F
:10762900E012BC53D8F67920E030E702792F3048D0
:107639000A12096D14651070027923E97E1812BCCB
:1076490053E51230E70A908C627E20126615800A93
:107659007E20E51112766D125F010510C3E558957C
:1076690010509C2264B4602464B475F03284C0F074
:1076790012BC40CE2404CED0E075F00584C0F012CF
:02768900BC4003
:10768B00CE2404CED0E02302BC4090769B0266153C
:10769B002D2D2D000140FFFFFFE0FFFFFFFFC2502C
:1076AB0020093C301239202836E558F46031D2508D
:1076BB00E559F5103033066558600205101276EE69
:1076CB0012773375A7049006DCE512F0E511F0E5AF
:1076DB0017F0E510F075A7049006E0ECF0EBF075F1
:1076EB00A7002275A704758307125D5B7813E0F67C
:1076FB0008B819FA9006D07811E6F008B819FAE52F
:10770B001CF516F0E51BF515F0758306E5102354F3
:10771B001E24B0F582E0F513E0F5149006DAE514BB
:10772B00F0E513F075A700221206D8E5BD75F0053C
:10773B00A485F012F511E4F519FEF51CF51D12A840
:10774B00A9C23DC2567F3C12B4F2303D05751900FB
:10775B008077DFF3E5596558700A301007EE24D3B4
:10776B005002D2568C1B8D1AE519FD24E250DEAE69
:10777B001CAF1D7C0012571EEFF51924F650CEAC32
:10778B001BAD1A12B42E20D1108E048F05E519757E
:10779B00F0A7A4AEF0FF12571EAC12AB117AA012D9
:1077AB005649EB33FBEC33FC20D11AEF9BEE9C508C
:0277BB0014C3F5
:1077BD00E51213FCE51113FBC3EF9BEE9C4004ACEB
:1077CD0006AB078C128B119006E2E519F0127817B3
:1077DD00AC16AB157AC8125620A912A8111257C4AF
:1077ED00ED7005EC249E50057C807B0822C3E57A64
:1077FD00305602E55C9513FFE55E305602E55D956A
:10780D0014FEC3EF9BFBEE9CFC22AE16AF157C0065
:10781D00E519FD24F6501A12571E7C007D061255EF
:10782D00FE7C007D0512571E8F10EEF51724E950D2
:10783D00037517FF2212B45912785F12789412B99A
:10784D00F91278BA2048091279421279720279D563
:10785D00806630480E7F177E1A746A305F02746737
:10786D0012BC8575A7049006D07811E0F608B819FA
:10787D00FA7F187E007812751906E60812BC53EED1
:10788D002404FED519F42275A7049006D8E0F51648
:10789D00E0F515E0F514E0F513E0F512E0F511E073
:1078AD00F517E0F510E0FCE0FB75A700227F187ED0
:1078BD0026AC14AB1302BA879006E4E0F51CA3E0E6
:0D78CD00F51B7F2A304E089091FE1265CA0F
:1078DA0080220F9091B11266139004EEE0FEF51E1D
:1078EA00A3E0FFF51FEE24E950047E177F6F12799B
:1078FA005312791A75172A751627125E7020240CEE
:10790A00205F0C7F2B7E23743F02BC53205FF4223E
:10791A00AC1CAB1B7A48305D027A27125620A91E8E
:10792A00A81F1257C4ED4C60027BFF7F207E28EB14
:10793A0012BB947E39027E9F7F2B908F9912661319
:10794A00E517F46022AE17AF107C007D3C12572B6E
:10795A00A805EF7F2A7E0C12BB8E7E16743B12BCE2
:10796A00817E18E812BB8822AE12AF117C007D0A14
:10797A0012572BA805EF7F207E3012BB8E7E3A74F9
:10798A002C12BC857E3CE812BC6B0F7E2974450222
:10799A00BC53746C8007746E205602746D7E291273
:1079AA00BC85301707742D7E3A12BC85227C007D77
:1079BA000A12572BA805EF7F2A7E3012BB8E7E3A19
:1079CA00742C12BC857E3CE802BC6B127AF6E54840
:1079DA0024F650051279B780B9E559046558600D47
:1079EA001279B712799CE559655860AA22A21792B2
:1079FA003D8E1E8F188515179006D0E0F511855813
:0E7A0A001015101237BBC3E51195105002F491
:107A180004F924A65005C374B399F9E975F00584EF
:107A2800F924EE50027911907B36E993F5F01206AD
:107A3800E2E5BD23A4A9F0E51B2517FDE51C3516D5
:107A4800FEC3ED99F515EE9400F51675A70075833C
:107A580006E55823541E24B0F582E0A3F513E0F59B
:107A680014127AF6203D242017211206D8E5BD7598
:107A7800F007A4FB9518E5F0951E400FEB9FE5F085
:107A88009E4008EF9518EE951E500EA23D9217AE37
:107A98001EAF181279B702799C306B10127A93E5F1
:107AA8003F20E007746D7E2212BC852275A70090E6
:107AB80006E0E516F0A3E515F01279B71279A0747F
:107AC8006C7E2312BC858558101276EE12785F12F0
:107AD80078948C168B151278BA1277DD1276E0122C
:107AE800B9F99006E2E0F519127817027942C3E570
:107AF8007A305602E55C9513FFE55E305602E55D87
:107B08009514FE92175003125895AC16AB157AC807
:107B1800125620A906A8071257C47E037FE7ED7006
:107B28000CEB2418EC34FC4004AE04AF032200171D
:107B38002E43576C8092A4B6C5D3DFE6EDF3F8FD6B
:0D7B4800305E4F30504C75A7009006E0E015
:107B5500A3FCE0FBECA2E79217402024FE50047F33
:107B65003B8022AE04AF037C007D1412572B745466
:107B75002F2017029F9FFF7462800C1258A5EC24DA
:107B8500FE50E07F6D743D7E0012BC537E017D1971
:107B95007C03127B9B227F3D12C6AAEF2DFFDCF8EA
:107BA50022E534243750012212C76512C37D12B86D
:107BB5001912B8B5127D1F12B2BA12BDC312C6454D
:107BC500127D77125D737F207E2B12B94D12C2553F
:107BD50012C2CD127C58122CD602C5AFE579FD2410
:107BE500A050027D5FED24CD401E744520750C2DFF
:107BF500FFF512127C2D1FBF44F922C39DFFF5121C
:107C0500127C2D0FBF46F92220750EED2413FFF5CA
:107C150012127C2D0FBF78F922C374779DFFF512E0
:107C2500127C2D1FBF12F922EF24BA40082433FC21
:107C3500C374329C1404FC24D750047C238009ECC3
:107C45002375F005842413FC7E0512C6AA0EECB537
:107C550006F822127BE17F457E047D0E12C6AA0E30
:0F7C6500DDFA7F437E00746412BC537F4F7D12A3
:107C7400127D087F3B7D12127D087F597D16127D8F
:107C8400087F317D16127D087F637D1A127D087F7F
:107C9400277D1A127D087F6D7D1E127D087F1D7D54
:107CA4001E127D087E057F1912C6AA0FBF72F978CD
:107CB40004E57924CD50027809E8305C0123F87F8B
:107CC4001B127CF77F6B127CF718305C01187F2540
:107CD400127CF77F61127CF718305C01187F2F1239
:107CE4007CF77F57127CF718305C01187F39127CBF
:107CF400F77F4D7E00E875F00A847004E802BC400A
:107D0400E802BBDBEF6512600C7E04EE20E0071294
:107D1400C6AA0EDDF62212C6DA80F79090667F2896
:107D24007E2C1266157E3B12BA9EAC5EAB7A7F3017
:107D34007E19C23D12BADD908F9D7F5D7E2D126645
:107D44001578B9C3E57A9618FBE55E96FC7F507EFC
:107D540019D23D02BADDE51164B4700122E51112B5
:107D6400C5067831790F7D0B12C5F81F1E907E076A
:107D740002BCB3E5716012E57012C5067831790F63
:107D84007D0412C5F40DBD0AF97F01127DDF7F1D4C
:107D9400127DDF7E23127DE97E3F127DE97E247F02
:0F7DA40017127DF37E397F02127DF37E247F0755
:107DB300127DFD7E397F1C127DFD7E317F0212C64E
:107DC300AA7F1C12C6AA7F0F7E2412C6AA7E3E1269
:107DD300C6AA7F0C7E2E90C19602BCB37E2A12C621
:107DE300AA0EBE39F9227F0812C6AA0FBF17F922BD
:107DF3007D0612C6AA0E0FDDF9227D0612C6AA0E53
:107E03001FDDF9220303E0A0E012B4597F18908A22
:107E1300A71266137F217E01744112BC537F2A7E11
:107E230001745312BC539005BEE0F51AA3E0F51993
:107E3300A3E0F51EA3E0F51D851A1C85191B751714
:107E430020127EBCE519251DF51BF51DE51A351E0F
:107E5300F51CF51E751729127EBC9005BA127EAC6F
:107E6300AC1AAB19751720127E7A9005BC127EAC42
:107E7300AC1EAB1D751729EC7006EB249B40012249
:107E83007A48305D027A271256201257C4ED4C60AF
:107E93000122AF177E07EB12BB3A7E1A0F90913384
:107EA300305D03909136026615E0FEA3E0FD12AA51
:107EB30003C3EB9DF8EC9EF922751627126030126E
:107EC3005ECAAF170F7E37909139305D0390913CB6
:107ED30002661512AA0375A7049005B478737F068A
:087EE300E6F008DFFBECF0EB18
:107EEB00F0E0E0E0FCE0FDE0FEE0FFEF2DFFEE3C1C
:107EFB009005C0F0EFF0801275A7049005BAE0FB77
:107F0B00E0CBF0EBF0E0E0E4F0F075A7002275A712
:107F1B00049005B478647F06E0F608DFFB75A700D4
:0E7F2B001260579005BEE51CF0A3E51BF02286
:102D6E00D23C799E770012A8A9E4F510F511F51260
:102D7E00F513F514F515F516F517C23D123085202D
:102D8E003D1F123085203D19E51F30E51130E40E50
:102D9E00122DE1303C08799EE724F5500122D51022
:102DAE00DBAE14AF157C00AD121256F88F55AE1671
:102DBE00AF177C00AD1312571E12591F7E00E5553A
:102DCE0030E7011E2DFFE43E30E7027F00740A2F2C
:102DDE00F55622C235E51CAF1DBFFF050FD235F4E7
:102DEE0004FABF003F752C00E518AF19BFFF050FA1
:102DFE00D262F404BF002D20E72A205B0123FF24BA
:102E0E00AA4021E51AAE1BBEFF050ED261F404BE28
:102E1E0000128547F0A4E5F020E709205B0123FEB0
:102E2E0024AA5001227C807B80305166302163C001
:102E3E0006C0078AF0E545A4AEF0FFE556205B011B
:102E4E001375F009A4ACF0FD12571E74FFBE0001FD
:102E5E00EFFA24C050027A3FD007D006E55212C5D1
:102E6E0006303504B2D5B2D1EA8CF0A430E70205B3
:102E7E00F0748025F020D10495F095F0FCEA8BF0EB
:0A2E8E00A430E70205F0748025F07F
:102E980030D50495F095F0FBC3EC2F2062029F9F7C
:102EA800FFEB2E3061029E9EFE200C05122F39404A
:102EB80020EF2460401B243F5017EE24604012246A
:102EC8003F500EEF24D6FFEE249FFE303C04799E3F
:102ED800072212C6AAE51E24FB50F60E12C6AAE562
:102EE8001E24F650EC1E1F12C6AAE51E24F150E15E
:102EF8001E0F12C6AAE51E24EC50D60F12C6AAE56C
:102F08001E24E750CC1F1F0E0E12C6AAE51E24E28F
:102F180050BF1E0F0F12C6AAE51E24DD50B30E12B5
:102F2800C6AAE51E24D850A91E1E1F1F02C6AAD372
:102F380022C261EE10E706D2E7F404D261FE24D380
:102F480040EDD262EF10E706D2E7F404C262FF2434
:102F5800D340DCC260EFB506005003CED260FF2438
:102F6800FD50CC903003938EF0A4AAF033CA33CA34
:102F780033CA33CA33CA33FA90302D938FF0A4334F
:092F8800C5F033CA90304E93FBF2
:102F9100122FCB9570500224B412C506EA8BF0A40F
:102FA10030E70205F0C3748095F020D50425F025A3
:102FB100F0FEEA8CF0A430E70205F0C3748095F0CE
:102FC10030D10425F025F0FFC322E52C540723C39B
:102FD100902FD573800E800E8024801E8010800A71
:102FE10080108012EB22742D9B22742D2B22745A97
:102FF1009B22745A2B2274879B2274872B2274B3D1
:103001009B22FFFFCCAA928071665D554E494440D8
:103011003C383533302E2C2A282725242322212001
:103021001F1E1D1C1B1A1A1918181717818181825E
:1030310082838384858687898A8B8D8F90929496EB
